:020000040800F2
:20000000600800200D0E0008E10B0008E30B0008E50B0008E70B0008E90B0008000000005D
:20002000000000000000000000000000EB0B0008ED0B000800000000EF0B0008990B000814
:200040004D0E0008510E0008550E0008590E00085D0E0008610E0008650E0008690E000818
:200060006D0E0008710E0008750E0008790E00087D0E0008810E0008850E0008890E0008F8
:200080008D0E0008910E0008950E0008990E00089D0E0008A10E0008A50E0008A90E0008D8
:2000A000AD0E0008B10E0008B50E0008B90E0008BD0E0008C10E0008C50E0008C90E0008B8
:2000C000CD0E0008D10E0008D50E0008D90E0008DD0E0008F10B0008E50E0008E90E00088B
:2000E000ED0E0008F10E0008F50E000810B586B025208DF8040001208DF8050000208DF8D2
:20010000060001208DF8070001A800F045F901214FF4804000F0BDF90121092000F0B9F99D
:200120000121042000F084FA4020ADF8000003208DF8020018208DF803008C4C00A92046B5
:2001400000F011FA8020ADF8000004208DF8030000A9204600F007FA4FF416500290002058
:200160000390ADF81000ADF814000C20ADF812007F4C02A9204600F099FA012240F2255171
:20018000204600F0E9FA002240F22771204600F0E3FA0121204600F0D5FA06B010BD38B550
:2001A000744801210170744C2078032832D140F20321204600F06EF894F8031294F8042205
:2001C00002EB012189B2884220D16C480121017060786B4901EB40206A4D2860810AC9B2B6
:2001E000800507D1084600F03CF804281CBF182000F06AF84FF40072E11C284600F018F87F
:20020000042801D0182002E0062000E01520BDE8324059E004280AD1E078002807D1207944
:20022000022804D100F065F857480121017031BDF8B504460D461646042700F0F3FA760826
:2002400007D035F8021B206800F016FB0746042F01D03846F2BD2068801C2060761EF0D17D
:20026000F7E770B504460D1B01D4042C01D2022070BD00F0D7FA0026A00200F1006420469E
:2002800000F0DBFA0428F3D1761C04F58064B542F5D270BD30B4002299B141F22103491E41
:2002A00010F8014B82EA042292B208245500120446BF83EA050292B2AAB2641EF6D10029F2
:2002C000EDD1104630BC704710B5304C20702A48417861708078A07003212046FFF7DAFF39
:2002E0000112E17020712A48002101702948052133E010B5254C062020701F48417861707E
:200300008078A07003212046FFF7C4FF0112E1702071462060714320A0711620E07121202A
:200320002072002060720620A0724620E072492020734E2060734920A0735320E073482062
:2003400020740C21601DFFF7A5FF01126174A0740F48002101700F4813210170012240F28F
:2003600027710348BDE8104000F0F6B9000C01400038014017000020180000205704002056
:20038000000E0008500400205604002028040020550400205804002070B403781A460121F7
:2003A000C478ECB1164B1B6803F4E063C3F5E0631B0A4478C3F10405AC4085780F2626FA6F
:2003C00003F32B4023431B010E4C1355007842110D4B00F01F0001FA00F043F8220006E018
:2003E00050110A4A03F01F03994042F8201070BC7047074A114008430649086070470000B2
:020000040800F2
:200400000CED00E000E400E000E100E080E100E080FFFF1F08ED00E010B427490A6802F033
:200420000C02082A18BF254A0ED10A680B68C2F38342921CDB0358BF214B04D50B689B03FF
:200440004CBF1F4B1D4B5A4302600B681D4A0468C3F303139B5C24FA03F343600B684468E1
:20046000C3F302239B5C24FA03F383600B684468C3F3C2239B5C24FA03F3C3600968C3682F
:20048000C1F381318918097CB3FBF1F1016110BC70470D4A0029116814BF084321EA000039
:2004A00010607047094A0029116814BF084321EA00001060704700000410024000127A00EE
:2004C00000093D0000000020181002400C10024080B56E49884206D101210420FFF7E2FF44
:2004E000002104203CE06A49884206D101210820FFF7D8FF0021082032E06649884206D185
:2005000001211020FFF7CEFF0021102028E06249884206D101212020FFF7C4FF00212020A5
:200520001EE05E49884206D101214020FFF7BAFF0021402014E05A49884206D101218020C9
:20054000FFF7B0FF002180200AE05649884209D101214FF48070FFF7A5FF00214FF48070C5
:20056000FFF7A0FF01BD2DE9F041CB7803F00F02DB0644BF8B781A430B88DCB22CB3D0F88E
:2005800000C0002401250F2605FA04F7BE460EEA0308F04514D14FEA840E06FA0EF82CEA1A
:2005A000080C02FA0EFE4EEA0C0C91F803E0BEF1280F08BF476103D0BEF1480F08BF076106
:2005C000641C082CE0D3C0F800C04FF48074A34228D3D0F804C0002401250F2604F1080716
:2005E00005FA07F7BE460EEA0308F04515D14FEA840E06FA0EF82CEA080C02FA0EFE4EEAA1
:200600000C0C91F803E0BEF1280F08BF476191F803E0BEF1480F08BF0761641C082CDDD3FC
:20062000C0F804C0BDE8F081016170474161704770B41D4A00284CBF94691468C0F3034584
:2006400083B200F44016B6F5401F06D124F07064156825F0706515600CE0C60244BF032696
:2006600006FA05F503D4450D2D0103FA05F5AC4344F0706421B1410D090103FA01F10C43D3
:2006800000284CBF9461146070BC704700080140000C014000100140001401400018014046
:2006A000001C0140002001400400014030B585B004460D46208A4CF6FF710840E988084320
:2006C0002082A0894EF6F3110840A98808432989084369890843A081A08A4FF6FF410840F1
:2006E000A9890843A08200A8FFF796FE144884420CBF03980298296819225043A289120467
:200700004CBF49008900B0FBF1F16422B1FBF2F00001030902FB1311A3891B0406D5C9003E
:200720003231B1FBF2F101F0070105E009013231B1FBF2F101F00F010843208105B030BD5E
:20074000003801400029818912BF41F400514DF6FF7211408181704710B40B065B0F012474
:2007600001F01F0104FA01F1012B08BF0C3003D0022B0CBF10301430002A026814BF11433F
:2007800022EA0101016010BC7047C905C90D818070478088C005C00D704700880140481E8B
:2007A0008041C043C00F704710B40A06520F012301F01F0403FA04F4012A08BF828903D0BD
:2007C000022A0CBF028A828A2240090A03FA01F10088084022B1401E8041C043C00F00E0B2
:2007E000002010BC70470122090A02FA01F189B2C9430180704710B450F8041B81B10268EC
:020000040800F2
:200800001218001D50F8043BDC0744BFA9F10104E31852F8044B43F8044B091FF9D1EBE7A3
:2008200010BC704700E00000DFF8A800DFF8A8100160DFF8A8100160704738B505464FF4C4
:20084000302000F051F8042815D1DFF89440206840F0020020606560206840F040002060DB
:200860004FF4302000F040F8052804D0216841F6FD721140216032BD70B504460D464FF4C7
:20088000005000F031F8042810D1154E306840F00100306025804FF4005000F025F80528B4
:2008A00004D0316841F6FE721140316070BD0D480168C90701D5012070470168490701D54A
:2008C000022070470068C00601D5032070470420704700000420024023016745AB89EFCD60
:2008E000102002400C20024010B5FFE70446FFF7DEFF03E02CB1FFF7DAFF641E0128F9D04D
:2009000004B9052010BD50F8041B61B150F8042BD30744BFA9F101039A18002342F8043B6F
:20092000091FFAD1EFE77047F0B58BB001A80FF2A811242200F0EFF800214FF00060FFF721
:2009400058FD00F086F8FFF7D1FB00F00FF94FF4167000F01BF900F01CF90028FBD0222112
:2009600001A8FFF797FC01128DF826108DF8270003244A4D01AE242731782846FFF705FF02
:2009800080212846FFF709FF0028F9D0761C7F1EF2D1641EEED100F0FCF80128FBD10A2023
:2009A00000F0F4F83E4C2068401C20603D4D2968401A33280CD33C48007848B914223B4907
:2009C0003B4800F09BF83B4800210180FFF7E7FB20682968401AB0F5167F02D936480021ED
:2009E000017036488178491C81700278C9B291420ED100218170417881F0010141703048AB
:200A000019B10421FFF710FE02E00421FFF70EFE2C48017839B1491C0170C9B2652902D34F
:200A200025480021017020686528B4D3224800780028B0D124480168244A1140B1F1005FFB
:200A4000A9D141680091009C006800F0C5F8A047A1E710B582B001210C20FFF71AFD01214E
:200A60000120FFF716FD01211948FFF7E1FD01211848FFF7DDFD124C2046FFF729FD04209F
:200A8000ADF8000001208DF8020010208DF8030000A92046FFF767FD13BD0000003801409F
:200AA000480400204C04002017000020200200201800002046040020570400201400002090
:200AC000000C014056040020001000080000FE2F000430000002300046431621001C064E74
:200AE0004F57535F4543555F5A5F424C5F4C535F56332E305F312E302E3200004AB38B07FA
:200B000007D0521E11F8013B00F8013B21D08B07F7D183071ED1103A07D330B4B1E8381068
:200B2000103AA0E83810F9D230BC530724BFB1E80810A0E8081044BF51F8043B40F8043B54
:200B4000D20724BF31F8022B20F8022B44BF0B7803707047083A07D3B1E80810083A40F847
:200B6000043B40F804CBF7D25307E4E7174847F6FF4141601649F0220A70002181600721AF
:200B800001607047481E8041C00F704711490881704710480189F5E70E48018909B1491E37
:200BA0000181418811B14188491E4180818811B18188491E8180C18811B1C188491EC180FF
:200BC000018809B1491E01807047000010E000E023ED00E03C04002080F3088870477047A2
:200BE0007047FEE7FEE7FEE7FEE7704770477047F0B581B0284C40F2255529462046FFF7C4
:020000040800F2
:200C0000D3FD60B3254826490968016025480021017029462046FFF7E6FD2046FFF7B9FD84
:200C2000214B1A8821495054214DC0B2012805D12E78032E02D11F4E012737702870501CCF
:200C4000188040F2052280B2904208D31A4D2870002018801948FFF751FFFFF7A0FA40F2A4
:200C6000277529462046FFF79FFD98B1144E30781449415C2046FFF788FD3078401C30709F
:200C800011490978C0B2884204D1002229462046FFF762FD01B0F0BD003801404C040020D5
:200CA00048040020170000204604002020020020590400205704002054040020180000203D
:200CC0005504002028040020580400202648016841F0010101604168244A114041600168F6
:200CE000234A11400160016821F480210160416821F4FE0141604FF41F018160016821F435
:200D0000803101601B490A6842F010020A600A68920892000A600A6842F002020A6041687A
:200D2000416041684160416841F480614160416821F47C114160416841F460114160016823
:200D400041F08071016001688901FCD54168890889004160416841F002014160416801F0D0
:200D60000C010829FAD17047001002400000FFF8FFFFF6FE0020024010B5084979441C31F6
:200D8000074C7C441A34A14206D0081D0A68511888470146A142F8D110BD00BF08000000E3
:200DA0002800000063FBFFFF44040000180000200000000043FAFFFF180000003C0100009F
:200DC000000000200000000000F009F8002801D0FFF7D2FF0020FFF7A7FD00F002F801207D
:200DE000704780B500F002B800BF00000746384600F002F8FBE7000080B5C046C046024A7A
:200E000011001820ABBEFBE7260002000148804701480047CD0C00081D0E0008C046C04656
:200E2000C046C046FFF7D0FFFFF7DABEFFF7D9BEFFF7D8BEFFF7D7BEFFF7D6BEFFF7D5BE9C
:200E4000FFF7D4BEFFF7D3BEFFF7A6BEFFF7FEBFFFF7FEBFFFF7FEBFFFF7FEBFFFF7FEBFAA
:200E6000FFF7FEBFFFF7FEBFFFF7FEBFFFF7FEBFFFF7FEBFFFF7FEBFFFF7FEBFFFF7FEBFDA
:200E8000FFF7FEBFFFF7FEBFFFF7FEBFFFF7FEBFFFF7FEBFFFF7FEBFFFF7FEBFFFF7FEBFBA
:200EA000FFF7FEBFFFF7FEBFFFF7FEBFFFF7FEBFFFF7FEBFFFF7FEBFFFF7FEBFFFF7FEBF9A
:200EC000FFF7FEBFFFF7FEBFFFF7FEBFFFF7FEBFFFF7FEBFFFF7FEBFFFF7FEBFFFF7FEBF7A
:200EE000FFF786BEFFF7FEBFFFF7FEBFFFF7FEBFFFF7FEBFFFF7FEBF00000000010203042F
:200F000001020304060708090204060814000001FFFFFFFFFFFFFFFFFFFFFFFFFFFFFFFF90
:200F2000FFFFFFFFFFFFFFFFFFFFFFFFFFFFFFFFFFFFFFFFFFFFFFFFFFFFFFFFFFFFFFFFD1
:200F4000FFFFFFFFFFFFFFFFFFFFFFFFFFFFFFFFFFFFFFFFFFFFFFFFFFFFFFFFFFFFFFFFB1
:200F6000FFFFFFFFFFFFFFFFFFFFFFFFFFFFFFFFFFFFFFFFFFFFFFFFFFFFFFFFFFFFFFFF91
:200F8000FFFFFFFFFFFFFFFFFFFFFFFFFFFFFFFFFFFFFFFFFFFFFFFFFFFFFFFFFFFFFFFF71
:200FA000FFFFFFFFFFFFFFFFFFFFFFFFFFFFFFFFFFFFFFFFFFFFFFFFFFFFFFFFFFFFFFFF51
:200FC000FFFFFFFFFFFFFFFFFFFFFFFFFFFFFFFFFFFFFFFFFFFFFFFFFFFFFFFFFFFFFFFF31
:200FE000FFFFFFFFFFFFFFFFFFFFFFFFFFFFFFFFFFFFFFFFFFFFFFFFFFFFFFFFFFFFFFFF11
:020000040800F2
:20100000900800203D830008F97F0008FB7F0008FD7F0008FF7F00080180000800000000BB
:20102000000000000000000000000000038000080580000800000000078000088D61000813
:201040007D8300088183000885830008898300088D830008918300089583000899830008E0
:201060009D830008A1830008A5830008A9830008AD830008B1830008B5830008B9830008C0
:20108000BD830008C183000809800008C9830008CD830008D1830008D5830008D98300085F
:2010A0004180000881800008E5830008E9830008ED8300083F3C0008F5830008F98300087B
:2010C000FD8300080184000805840008098400080D840008978000081584000819840008D7
:2010E0001D84000821840008258400082DE9F0439DB04FF4004001F0ACFC0121012001F003
:20110000EAFC01211D2001F0EFFC01214FF4007001F0EAFC01214FF4806001F0E5FC0121C9
:201120004FF4006001F0E0FC01214FF4806001F007FD00A801F0BCFDFF20ADF800000020CF
:201140008DF80300DFF8704D00A9204601F04FFD00A801F0ADFD0320ADF8000000208DF877
:201160000300DFF8E08D00A9404601F040FDDFF84C5D284601F0FAFDDFF8440D1290DFF854
:20118000E86D06F238001390002014900520159000201690802017904FF4007018904FF4EE
:2011A0000067199720201A9000201B901C9012A9284601F045FE0121284601F05CFEDFF8A8
:2011C000885D284601F07EFE0BA802F07FF80020ADF82C002020ADF82E004FF4FA60ADF8ED
:2011E00030004FF48079ADF8329001208DF834000BA9284601F02DFF02A802F070F860207F
:20120000ADF808000120ADF80A000420ADF80C004FF47A70ADF80E000020ADF8100008209F
:20122000ADF812000020ADF81400ADF8169002A9284601F04BFF02A9284601F083FF02A948
:20124000284601F0B5FF00A801F032FD4FF4E060ADF8000018208DF8030003208DF8020021
:2012600000A9204601F0C3FC4FF46040ADF8000018208DF8030003208DF8020000A940468E
:2012800001F0B5FC4FF4E061204601F028FD00A801F00EFD4FF48054ADF8004004208DF863
:2012A000030000A9404601F0A2FC02A802F017F87020ADF808000120ADF80A000020ADF8F0
:2012C0000C0040F2CF70ADF80E000020ADF810000820ADF812000020ADF81400ADF8169006
:2012E00002A9284601F09BFF0821284602F020F80821284602F023F80821284602F027F85D
:201300000821284602F02AF8ADF838704FF48060ADF83A00ADF83C902020ADF83E00ADF89A
:2013200040400020ADF84200ADF844000EA9284601F0BEFF2021284602F018F880212846AA
:2013400002F025F801228021284601F0E7FF0121284601F0CEFF288B48F68F710840F0837B
:20136000A88B4FF68F71084030840121284601F0DDFF0121284602F009F800220121284667
:2013800001F0CCFF00221021284601F0C7FFDFF86C4C204601F0FEFFDFF8645C284601F040
:2013A000F9FF0121204602F043F80121284602F03FF806A802F033F84FF480300690012052
:2013C0008DF81C0000208DF81D004FF460260896099705208DF8280006A9204602F001F8D1
:2013E00006A802F01CF801208DF81C0000208DF81D000896099701208DF8280006A928468C
:020000040800F2
:2014000001F0EFFF204602F02FF8284602F02CF8204602F02EF80646284602F02AF8064256
:20142000F6D100F06AF8022301220321204602F02FF8022302220921204602F029F8072392
:2014400003221021204602F023F8022304220821204602F01DF8022305221946204602F0DF
:2014600017F8012002F0AFF8022301220721284602F00EF80121204602F044F80121284687
:2014800002F040F80121204601F0DBFF0121284601F0D7FF4FF4A06002F0B6F812208DF8DE
:2014A000040001208DF8050000208DF8060001208DF8070001A802F0ACF819208DF8040024
:2014C00001208DF8050000208DF8060001208DF8070001A802F09DF818208DF804000020F8
:2014E0008DF805008DF8060001208DF8070001A802F08FF81DB0BDE8F08370B5DFF8FC4AE1
:2015000000224FF49061204601F0A5FFDFF8585A0020E8816882E8824FF4E041204601F059
:20152000FAFFDFF8DC6A4FF4E041304601F0F3FF0121204601F0F8FF0121304601F0F4FFEC
:201540000321204602F02AF8002301222979204601F0FCFF002302226979204601F0F6FF3E
:2015600000230322A979204601F0F0FF0421204602F047F80121204601F0DFFF102604214D
:20158000204602F037F80028F9D01421204602F00DF8E989001D01EBE000E88118212046DE
:2015A00002F004F8698A001D01EBE00068821C21204601F0FBFFE98A001D01EBE000E88223
:2015C0000421204602F01DF80121204601F0B5FF761ED4D1E8892882688AA882E88A2883BF
:2015E0004FF48051204601F096FFBDE87040F8B5DFF8544900220121204601F08FFEDFF876
:20160000FC5900224FF49061284601F024FF0021284601F089FF0421284601F0F2FF0121FE
:20162000284601F0BBFFDFF8D8690121304601F0B5FF00F029F800F042F9DFF82C79002361
:2016400001227979284601F081FF002301223979304601F07BFF0021284601F065FF0421B4
:20166000284601F0CEFF01224FF49061284601F0F2FE0121204601F089FE012201212046ED
:20168000BDE8F84001F04ABE2DE9F04F85B0DFF8D808C08AADF80800DFF8CC18C98902AA83
:2016A0005180DFF8C4385B8A9380D080ADF810105381DFF89448208C4DF6FF7108402084A7
:2016C000DFF840094FF4A06101804FF46040ADF8000018208DF8030003208DF8020000A98A
:2016E000DFF8600801F083FA0025DFF81C09019002AEDFF818794FF00308DFF80099208C0D
:201700004FF6AA2108402084208B48F68F7108402083A08B4FF68F710840A08300230122D8
:2017200001980178484601F011FF0023012201984178DFF8CC0801F009FF0121204601F053
:2017400025FE0121204601F01AFE0028F9D00121484601F0E9FEDFF81008C08B3988084316
:201760002083DFF80408008C79880843A083208CB988084320840121204601F0C4FD0421AD
:20178000484601F03EFF0421484601F033FF48B98021204601F0F3FD20B9DFF8740800683A
:2017A0008005F0D50021204601F0ADFD0021484601F0BAFE1421484601F0F8FE3188D1EB46
:2017C0004000824648BFCAF1000A1421DFF8300801F0ECFE7188D1EB4000834648BFCBF195
:2017E000000B8021204601F0CAFD012804D0DFF82008006880051DD5DFF8180800780028AD
:020000040800F2
:201800000CBF10204FF4007001F07DFFDFF80808002101704FF46040ADF8000018208DF8EF
:20182000030003208DF8020000A9DFF8180701F0DEF941E041F23D30824501DA83450CDB82
:201840008021204601F0A2FDDFF8C8070078002814BF4FF400701020D6E7BBF15C0F04DA43
:2018600002F0EEF90A28B8BF6D1C07F20607361D0198801C0190B8F101087FF440AFDFF853
:20188000E806C08B46F2600108432083DFF8D806008C40F06000A083208C40F255510843C5
:2018A0002084ADB2022D07D3DFF86407006840045CBF202001F027FF05B0BDE8F08FDFF80C
:2018C0005C074FF47A7101808180018140F2CF718181DFF8940600214183C170DFF8841C01
:2018E00000220A800285704781B0DFF87C064178491E052944D8DFE801F0142C2C030314CC
:20190000C189DFF81C271268A1EB420101F30F01ADF80010408ADFF8501C0968A0EB410017
:201920002AE0418ADFF8F8261268A1EB420101F30F01ADF80210DFF8301C0968C08AC0EB50
:201940004100BDF90210401A00F30F00ADF8000016E0C189DFF8C8261268A1EB420101F33B
:201960000F01ADF80010DFF8001C0968C08AC0EB4100BDF90010401A00F30F00ADF802003F
:20198000009801B070470000F0B50B4643F2206606FB00F7DFF8D42B5343FA1802EBD272EF
:2019A0005610DA1B02EBD2725710002E0BD5002F48BF4FF0050C11D4012BACBF4FF0030CD6
:2019C0004FF0040C0AE0002F58BF4FF0020C05D5012BB4BF4FF0060C4FF0010CDFF88825A1
:2019E00082F801C0B2F81AC0B2F91CE0BEF1000F08BF4FF0000C04D0BCF5FA6F38BF0CF1CF
:201A0000010CA2F81AC04FF0000C82F800C092F801C0ACF1010CBCF1050F65D8DFE81CF0FA
:201A200006007000C9000A016501A901181403EBD0304514D81B518BB1F5FA6F10D200EB2E
:201A4000D0704010011400EBD130401400F2E83189B2381407EBD03001EB6040441B06E04C
:201A6000011400EBD130411489B228460024C1F5FA639BB2B3F5A07F02DD40F2CF752BE0BC
:201A8000A62B0BDB01F24015ADB2B5F5FA6F23DB0123137040F69F735D1B1CE00D1A4FF40A
:201AA000A676ADB2B54214D2612B0FDA4FF4FA61C0F5FA639BB2A62B38BF40F22A7000F2D6
:201AC0004015ADB2B5F5FA6F06DBE1E740F28460401AA1F10D05ADB2136DDFF8946A33603B
:201AE000536DDFF8906A3360DFF88C3A1678002E1E8806BF4DF6FF773E4046F400567CE1DA
:201B0000301406EBD0304414508BB0F5FA6F11D2F01B00EBD0704010011400EBD130401491
:201B200000F2E83189B2381407EBD03001EB60400C1B06E0A1B2F019031400EBD3304014D3
:201B40000024C0F5FA639BB2B3F5A07F02DD40F2CF752CE0A62B0BDB00F24015ADB2B5F5D3
:201B6000FA6F24DB0123137040F69F735D1B1DE0451A4FF4A676ADB2B54215D2612B0FDA29
:201B80004FF4FA60C1F5FA639BB2A62B38BF40F22A7101F24015ADB2B5F5FA6F07DBE1E74F
:201BA00040F28461091A89B2A0F10D05ADB2D36C93E7301406EBD0304414508BB0F5FA6F7F
:201BC00011D2F01A00EBD0704010011400EBD130401400F2E83189B20C1B181403EBD030C1
:201BE00004EB604006E000216442981B031400EBD3304014C0F5FA639BB2B3F5A07FA6DCF5
:020000040800F2
:201C0000A62BA9DA051B4FF4A676ADB2B542CBD2612B0BDA4FF4FA60C4F5FA639BB2A62BBC
:201C200038BF40F22A7404F24015B4E740F284631C1AB9E7381407EBD0304014518BB1F5F4
:201C4000FA6F11D2D91B01EBD17149100C1401EBD431491401F2E83189B240181C1403EB92
:201C6000D433A0EB634405E00021FB1A1C1403EBD4335C14C4F5FA639BB2B3F5A07F02DD72
:201C800040F2CF752BE0A62B0BDB04F24015ADB2B5F5FA6F23DB0123137040F69F735D1BEA
:201CA0001CE0251A4FF4A676ADB2B54214D2612B0FDA4FF4FA64C0F5FA639BB2A62B38BF11
:201CC00040F22A7000F24015ADB2B5F5FA6F06DBE1E740F28460001BA4F10D05ADB2D36C60
:201CE000DFF88C683360136DFBE6381407EBD0304014518BB1F5FA6F11D2F11B01EBD1718B
:201D000049100B1401EBD331491401F2E83189B24018331406EBD333A1EB634408E0414283
:201D200089B20020BB191C1403EBD4335B145C42C4F5FA639BB2B3F5A07FA1DCA62BA4DA4C
:201D4000651A4FF4A676ADB2B542C5D2612B0BDA4FF4FA64C1F5FA639BB2A62B38BF40F24C
:201D60002A7101F24015AFE740F28461091B89B2B2E7181403EBD0304514F01A518BB1F5DC
:201D8000FA6F10D200EBD0704010011400EBD130401400F2E83189B2301406EBD030A1EB21
:201DA0006044281906E0011400EBD130411489B26C420020C1F5FA639BB2B3F5A07F3FF79C
:201DC0005CAEA62BBFF65EAE0D1B4FF4A676ADB2B542BFF47EAE612B0BDA4FF4FA61C4F5E3
:201DE000FA639BB2A62B38BF40F22A7404F2401567E640F284635C1A6BE61E8040F2D17612
:201E00008FB2B7422CBF518C518480B2B0422CBF908C9084A4B2B4422CBFD48CD4844FF47A
:201E200000364FF42037DFF8B0CA9CF900C0BCF1010F0ED1998218839C831D840420107175
:201E4000052050710620907130463E46118A938A0CE0988219839C831D8405201071042097
:201E60005071062090713846918A138A148BD064D4825382D1814FF4403050651665DFF83A
:201E8000D80A01210170F0BD80B55C4B0128986802BF40F400409860012009D020F40040A0
:201EA000986000224FF49061184601F0D4FA0020DFF8A81A087001BD000801400800024035
:201EC0004C24014038B54D4DDFF8904A2078012807D1A86840F40040A8600421284601F070
:201EE00090FB0121284601F0CAFA01F07AFDDFF8700A006843F63521884217D2DFF8640A6A
:201F00000078012815D1DFF8600A0078012810D06078401C6070C0B2052808D3002060700A
:201F20004FF40071DFF8440A00F0D5FE31BD0028F6D04FF40071DFF8340ABDE8344000F057
:201F4000CCBE0000000C0140002C0140DFF80C0A0078012805D1DFF8180A016821F4004121
:201F600001600120704700000000002038B500F059F8DFF8000A007801280CBF4FF4AF7328
:201F80001E23DFF8F40900884FF4C871884202D2332B28BF32231F480278DFF8E009418D81
:201FA000042A26D1B0F91C40DFF8D429B2F90050A54209DAB2F900505D19A542AFBF148004
:201FC00014881B19138014E0B2F90030A34210DB04F22C13B2F90050AB42BDBF1388A3F533
:201FE00096731380148034B9491CDFF898391B68125F418531BD0021FBE7000000240140A7
:020000040800F2
:2020000000280140402C0140902500087C250008BC030020680400206E040020342C0140A6
:202020003C2401402DE9F84FDFF85049DFF858190868C0EBC000228F1018C0080860DFF82F
:202040004C190A88824238BF0880DFF8443993F80090DFF840190988814228BF09F1010968
:202060005FFA89F9B9F1C90F28BF4FF0C80983F80090DFF82479386081422CBF4FF4807311
:202080008023DFF81899A9F80430DFF814391E68DFF810294FF496739E423ABF13885B1C4F
:2020A00000231380B4F92E30DFF8FCB8BBF900E0BEF1500FB8BF5B1C02DB012BA8BF5B1E5B
:2020C00040F2D1781BB24345A8BF4FF4FA63B4F93050BEF1460FB8BF6D1C02DB012DA8BF86
:2020E0006D1E2DB24545A8BF4FF4FA65258640F2E935AB420DDB81420BD3DFF8B0584FF054
:20210000050885F80080DFF8A8584FF0000885F800801288652A08D3DFF89828127822B99A
:2021200040F6B932904228BF3960B6F5967F0AD9DFF878281078042805D01078032802D004
:20214000481C38600023DFF86C683078012809D1DFF864080068A0F29110132802D2481CB9
:2021600038600023E38501F009FFDFF850184843C11300EB11400214608E3C2A03DA0428F6
:2021800003D2401C01E000B1401E6086A16B207AA0F13303DBB2092B08D2DFF81C381B6882
:2021A0004FF4C875AB4228BF4FF47A61DD2A0DDBDFF8E027128889B28A4207D340F6B93244
:2021C000914203D3DFF8E81701220A70618E042907D3DFF8EC17097819B9DFF8D4170022DC
:2021E0000A70DFF8CC8798F8001021B9627A012A08BF002002D0C82838BF401C2072617259
:202200003078012804BF012188F80010DFF85417097831B1DFF8A02712684FF4C8739A4261
:2022200002D2002288F80020A38EDFF89827128812B108B95B1C00E00023A386A38E152B0F
:2022400024BF002388F80030DFF838572B682B685B0440F19480B4F92C00C249B1F90010FA
:202260006FF0BC02914205DBDFF85C170968B1F55C5F05D96FF0770188422CDA78302BE03A
:20228000DFF8DC16096843F63522914218D389B2DFF838275118DFF83827514342F6AB220D
:2022A00091FBF2F16FF4F97209B29142A8BFDFF8241706DADFF81827914202DA114600E0FE
:2022C00000218142B8BF283802DB8842B8BF283000B2012800DB0020A085BBF9000000EB33
:2022E00080014800362190FBF1F080B23D28A8BFB4F92C0009DA012806DBB4F92C1048431A
:202300003C2190FBF1F000E0002098F8001001B90020DFF8C4160880B1F90000A083DFF89D
:20232000BC164FF400520A800021A170DFF87C76397801290ED100280CD5E079012805D196
:20234000022038702020A9F8040003E00120E07101F07AFC3878082809D03078002840F059
:20236000FE80DFF860060088002800F0F88001F034FA012840F0F38005203870EFE00023E0
:20238000A385DFF854B6ABF80030DFF808361B88D7F800C0634510D3DFF844361B8863B97F
:2023A000DFF840361B7843B9DFF83C361B78102B03D0DFF838361B78FBB1DFF8343693F906
:2023C0000030012B19D000B9BAB9B1B1DFF824A64FF40041504600F073FC01280DD0DFF833
:2023E00018060088C8214843DFF8CC150968DFF80C261268891A88422CD20020E071A0702B
:020000040800F2
:20240000DFF8A875387820B9012038700020A0830AE0B4F91C0038B10020A0838020A9F813
:2024200004000020ABF800003878082805D0307848B9DFF89005008828B101F0CEF90128C9
:2024400004BF0520387000F078FADFF890050021018084E02868400506D501F001FB18B9AA
:20246000286820F480602860286800050DD501F0F7FA30B14FF40041504600F021FC0128C6
:2024800003D1286820F400602860DFF820A59AF80000002863D000F050FADFF8F8040088BE
:2024A0003A68824238BF00230ED34BF26D239A4228BF4FF4804307D2131A9B034BF26C26B2
:2024C000361AB6B2B3FBF6F3DFF834653380DFF80C3536881E80824238BF40F29A2015D387
:2024E0004BF26C239A4228BF44F627600ED2461CB24208BF002009D0111A44F68D325143DE
:20250000181A80B2B1FBF0F000F29A2098F8001001B90020296840F67E72114209D040F290
:20252000046100B2884204DB40F20360DFF850140880A0839AF80000012810D128684004F0
:202540000DD4E079012806D102208AF800002020A9F8040003E00120E07101F075FBBDE85D
:20256000F18F00009A0000203C280140C0E0FFFF3824014038280140202C01404060500023
:2025800005016050400010055040600051000000060405060405000070B5DFF8C443206846
:2025A000DFF860140A88824238BF088044F2D15188420AD2DFF85014DFF8FC2312680A60E8
:2025C000DFF8481400220A7009E04AF2E921884205D3DFF83C14DFF8E02312680A60DFF89F
:2025E00030140968DFF8202412688A4206D2891A022903D2DFF8141401220A70DFF81414AF
:20260000081849F23E71884242D2DFF80004007800283DD1DFF86453E872A87A0A2825D315
:20262000DFF86003016841F480410160DFF8480300210180DFF8E003018841F001010180E5
:202640000020A883DFF8D40300210170DFF89C030170DFF894030078102804D0DFF88403B8
:202660000078012804D101F0D4FD01E0401CA872BE4EBC48007801284FF40071304602D11D
:2026800000F029FB01E000F028FBCD4800211DE0B948018842F2107291423CBF491C01800B
:2026A000B64D0020A872E87A0A2857D3B548016821F480410160DFF8600301884FF6FE720A
:2026C00011400180BE48017809B1491E0170AD48016801F48041AA6D02F48042914202D08F
:2026E000CF4901220A700068A865206843F6342188420DD29B480078012806D04FF4004113
:20270000BC4800F0DDFA012802D1C6480021017095480178012939D1C3490A88521C0A8032
:2027200092B2C24B1B78C82463439A4202DB002202700A80088828218C4E90FBF1F201FB2F
:20274000120014284FF40061304619DA00F0C3FA4FF40071304600F0BEFA21E0401CE872E8
:20276000C0B20928AED1924800780128AAD189480088894909688842A4D29148C821A5E717
:2027800000F0ABFA4FF40071304607E0774EA848007801284FF400613046DCD000F09DFAF0
:2027A000944C4FF40041204600F08AFA012809D1A048008840F2E33188429241D243D20F8F
:2027C0002A730FE0687B012808BF287399480088962838BF002004D340F25F11884201D3AA
:2027E000012028734FF40041204600F069FA68734FF40061204600F070FA4FF48061304607
:020000040800F2
:2028000000F06BFA4FF48051204600F066FA03F061F830B14FF40061204600F05CFA0020FC
:2028200053E062480178032902D00078042809D15848008858490968884203D25C480078D1
:20284000012817D04FF40041204600F039FA01282BD1287B48BB584800682821B0FBF1F2B1
:2028600001FB120014284FF48051204618D200F032FA17E0287B0128EDD14F4800682821C5
:20288000B0FBF1F201FB120014284FF48061304602D200F020FA01E000F01FFA022002E0FA
:2028A00000F01BFA0120012110E0287B012806D14FF48061304600F00EFA022005E04FF461
:2028C0008051204600F007FA012000215A4A11705A49087070BD00005901002010B5584842
:2028E0005849B1F9002003685A43B1F9021040684843D11302EB1141C21300EB124000142D
:2029000000EB214041F6CF4148434F49B1F90020C31300EB134002EB204000EBD07040105B
:202920000880164CE078401CE070C0B2022803D303F06DFA0020E07010BD80B512480068A9
:202940004CF2F111884204D3402000F0DCFE012002BD002002BD00006D0400206404002094
:20296000CC0300207704002078040020000C0140082401405F010020600400200000002053
:202980001C040020BC030020000400204C040020730400202C040020DC030020F802002084
:2029A000D00300203004002036040020680400207F0400207B040020C00300200071020052
:2029C0007E0400202A040020C4030020CCC5FFFF6CEEFFFF0CFEFFFF420400204004002067
:2029E00020040020700400205B0100206C0400206E0400200008014044040020E4030020A9
:202A0000A60300204E04002010040020870400200C040020CBC5FFFF4E01002069040020E2
:202A2000740400206F040020320400207904002076040020460400207D0400207C04002033
:202A400098030020B40300209A00002010430860704733490A6822F44042F7E710B4304917
:202A60000A6802F00C02082A18BF2E4A0ED10A680B68C2F38342921CDB0358BF2A4B04D534
:202A80000B689B034CBF284B264B5A4302600B68264A0468C3F303139B5C24FA03F343606E
:202AA0000B684468C3F302239B5C24FA03F383600B684468C3F3C2239B5C24FA03F3C36046
:202AC0000968C368C1F381318918097CB3FBF1F1016110BC7047164A0029116814BF084339
:202AE00021EA000010607047124A0029116814BF084321EA0000106070470F4A002911685B
:202B000014BF084321EA0000106070470B4A0029116814BF084321EA00001060704700001E
:202B20000410024000127A0000093D001401002014100240181002400C10024010100240A8
:202B4000044A0029116814BF084321EA0000106070470000042004E080B57C49884206D192
:202B600001210420FFF7C9FF002104203CE07849884206D101210820FFF7BFFF0021082047
:202B800032E07449884206D101211020FFF7B5FF0021102028E07049884206D101212020B4
:202BA000FFF7ABFF002120201EE06C49884206D101214020FFF7A1FF0021402014E0684982
:202BC000884206D101218020FFF797FF002180200AE06449884209D101214FF48070FFF7BF
:202BE0008CFF00214FF48070FFF787FF01BD2DE9F041CB7803F00F02DB0644BF8B781A43EA
:020000040800F2
:202C00000B88DCB22CB3D0F800C0002401250F2605FA04F7BE460EEA0308F04514D14FEA59
:202C2000840E06FA0EF82CEA080C02FA0EFE4EEA0C0C91F803E0BEF1280F08BF476103D0E6
:202C4000BEF1480F08BF0761641C082CE0D3C0F800C04FF48074A34228D3D0F804C0002499
:202C600001250F2604F1080705FA07F7BE460EEA0308F04515D14FEA840E06FA0EF82CEAEF
:202C8000080C02FA0EFE4EEA0C0C91F803E0BEF1280F08BF476191F803E0BEF1480F08BFCE
:202CA0000761641C082CDDD3C0F804C0BDE8F0814FF6FF710180022181700421C17070475F
:202CC000806802E0806880B270470140481E8041C043C00F7047016170474161704741F4C1
:202CE000803282618161826181698069704770B41D4A00284CBF94691468C0F3034583B289
:202D000000F44016B6F5401F06D124F07064156825F0706515600CE0C60244BF032606FAE4
:202D200005F503D4450D2D0103FA05F5AC4344F0706421B1410D090103FA01F10C430028C4
:202D40004CBF9461146070BC7047000000080140000C014000100140001401400018014087
:202D6000001C0140002001400400014001684908490001600021016041608160C16042493C
:202D8000884202BF4148016841F00F0156D04049884202BF3D48016841F0F0014ED03D4987
:202DA000884202BF3948016841F4706146D03A49884202BF3548016841F470413ED037491A
:202DC000884202BF3148016841F4702136D03449884202BF2D48016841F470012ED03149B6
:202DE000884202BF2948016841F0706126D02E49884202BF2D48016841F00F011ED02C49F2
:202E0000884202BF2948016841F0F00116D02949884202BF2548016841F470610ED026491F
:202E2000884202BF2148016841F4704106D02349884204D11D48016841F4702101607047C2
:202E400002681F4B1A408B681A430B6A1A430B691A434B691A438B691A43CB691A434B6AA9
:202E60001A438B6A1A430260CA6842600A6882604968C16070470029016812BF41F00101FA
:202E8000490849000160704708000240040002401C00024030000240440002405800024000
:202EA0006C0002408000024008040240040402401C0402403004024044040240580402400A
:202EC0000F80FFFF80B5DFF8A813884208D101214FF40060FFF711FE00214FF40060B5E0D8
:202EE000B0F1804F06D101210120FFF70FFE0021012014E0DFF87C13884206D101210220C4
:202F0000FFF704FE0021022009E0DFF86C13884209D101210420FFF7F9FD00210420BDE877
:202F20000440FFF7F3BDDFF85413884206D101210820FFF7EBFD00210820F0E7DFF8401356
:202F4000884206D101211020FFF7E0FD00211020E5E7CC49884206D101212020FFF7D6FDAD
:202F600000212020DBE7C849884208D101214FF40050FFF7C2FD00214FF4005066E0C3490A
:202F8000884208D101214FF40020FFF7B6FD00214FF400205AE0BE49884208D101214FF493
:202FA0008010FFF7AAFD00214FF480104EE0B949884208D101214FF40010FFF79EFD0021F6
:202FC0004FF4001042E0B449884206D101214020FFF79CFD00214020A1E7B049884206D12A
:202FE00001218020FFF792FD0021802097E7AC49884208D101214FF48070FFF787FD0021C3
:020000040800F2
:203000004FF480708BE7A749884208D101214FF48030FFF772FD00214FF4803016E0A24909
:20302000884208D101214FF40030FFF766FD00214FF400300AE09D49884209D101214FF492
:203040008020FFF75AFD00214FF48020FFF755FD01BD10B40388864A90420ED08A4CA042F2
:203060000BD0B0F1804F08D0824CA04205D0824CA04202D0814CA04204D14FF68F742340F7
:203080004C8823437E4CA04207D07E4CA04204D04FF6FF442340CC88234303808B888385B0
:2030A0000B88038590420BD0774A904208D07D4A904205D07C4A904202D07C4A904201D19B
:2030C000097A01860121818210BC704730B4028C4FF6FE731A400284048C8288038B4FF6C9
:2030E0008C752B400D882B434FF6FD752C400D892C434D882C435E4DA8420BD0624DA842EC
:2031000008D0684DA84205D0674DA84202D0674DA84210D14FF6F7752C404D892C434FF6CD
:20312000FB752C408D882C434FF6FF452A408D892A43CD892A4382800383C988818604848E
:2031400030BC704770B4028C4FF6EF731A400284048C8288038B48F6FF452B400D8843EABC
:2031600005234FF6DF752C400D894E88354344EA05143F4DA84202D0434DA84213D14FF60C
:203180007F752C404D8944EA05144FF6BF752C408D8844EA05144FF2FF352A408D89CE8925
:2031A000354342EA850282800383C988018733E070B4028C4FF6FF631A400284048C82889D
:2031C000838B4FF68C752B400D882B434FF6FF552C400D894E88354344EA0524244DA84292
:2031E00002D0294DA84213D14FF2FF752C404D8944EA05244FF6FF352C408D8844EA05241A
:203200004CF6FF752A408D89CE89354342EA051282808383C9888187048470BC704770B476
:20322000028C4EF6FF731A400284048C8288838B48F6FF452B400D8843EA05234DF6FF7534
:203240002C400D894E88354344EA0534084DA84202D00D4DA84205D14BF6FF752A408D8957
:2032600042EA851282808383C988A0F84010D3E7002C01400004004000080040000C00404B
:20328000001000400014004000340140004C0140005001400054014000180040001C0040AE
:2032A000002000400040014000440140004801400A884B881A438B881A43CB881A430B89A9
:2032C0001A434B891A438989114324E04FF6FF71818000210180C180418001727047002151
:2032E000018041808180C180018141818181C18170470029018812BF41F001014FF6FE72A0
:203300001140018070470029B0F8441012BF41F400414904490CA0F844107047002A82893E
:2033200014BF114322EA01018181704781827047028B4FF6F7731A40114301837047028B33
:203340004FF2FF731A4042EA012101837047828B4FF6F7731A40114381837047828B4FF264
:20336000FF731A4042EA01218183704782884FF68F731A4082808288114381807047008A2B
:203380000140481E8041C043C00F7047FFE7C9430182704780B59149884208D101214FF4F9
:2033A0000070FFF7AAFB00214FF4007016E08C49884208D101214FF48060FFF79EFB0021CB
:2033C0004FF480600AE08749884209D101214FF40040FFF792FB00214FF40040FFF78DFB22
:2033E00001BD4268804B1A400B681A430B7942EA0322426082687D4B1A40CB681A438B686A
:020000040800F2
:203400001A434B7942EA43028260C26A22F47002097C491EC9B242EA0151C16270470021A4
:203420000160017141718160C1600121017470470029816812BF41F0010149084900816026
:203440007047002981681ABF4FF48072114321F4807181607047C9B2002A426814BF11432D
:2034600022EA010141607047816841F004018160704780680006800E00F0010070470029E2
:20348000816814BF41F4A00121F4A0018160704770B4032407250A290AD3A1F10A0674436C
:2034A000C668A54026EA0505A3402B43C36007E04C430669A54026EA0505A3402B430361D2
:2034C00005231F24072A08D2521E5A43436B9440A34391401943416312E00D2A08D2D21F3C
:2034E0005A43036B9440A34391401943016307E00D3A5A43C36A9440A34391401943C16274
:2035000070BC70470029816814BF41F4801121F4801181607047826822F4E042114382687F
:203520008A4218BF816070470029816814BF41F4004121F40041816070470029816814BF22
:2035400041F4021121F402118160704770B4032407250A290AD3A1F10A067443C668A54070
:2035600026EA0505A3402B43C36007E04C430669A54026EA0505A3402B430361836BC3F380
:203580000154D21C121B521E02EB82021F249440A34391401943816370BC7047826B22F4E6
:2035A0004012491E42EA01518163704781B000220092009000982831081800900098006823
:2035C00080B201B070470A490028086814BF40F4000020F4000008607047000000240140C7
:2035E00000280140003C0140FFFEF0FFFDF7F1FF0824014000680140481E8041C043C00F06
:203600007047C943016070471B4908431B490860704770B403781A460121C478ECB1174B41
:203620001B6803F4E063C3F5E0631B0A4478C3F10405AC4085780F2626FA03F32B4023432F
:203640001B010F4C1355007842110E4B00F01F0001FA00F043F8220006E050110A4A03F082
:203660001F03994042F8201070BC7047074A114008430749086070470000FA050CED00E0CE
:2036800000E400E000E100E080E100E080FFFF1F08ED00E080B500F042FA02F06FFA00F046
:2036A00073FC00F0B6FDDFF81005C088DFF80C150880DFF80C1508800120FEF7E5FB0121AC
:2036C000DFF80005BDE80440FFF71DBEDFF8E804818843F6181251180904490C8161DFF8A1
:2036E000E80400210160704780B500F0B9F9022808BF4FF4006003D0012803D14FF4806047
:2037000000F001F801BD70B505464FF4167002F029FD0021DFF8AC04FFF7F5FDDFF8AC445A
:20372000206840F67E71084247D1022D24D0082D26D0102D1CD0202D16D0402D10D0B5F5D9
:20374000807F09D0B5F5007F1ED0B5F5806F23D0B5F5006F1CD023E0DFF8740409211EE06F
:20376000DFF86C0408211AE0DFF86404072116E0DFF85C04062112E0DFF8540405210EE0EF
:20378000DFF84C0404210AE0DFF84404032106E0DFF83C04022102E0DFF834040121C1704C
:2037A000DFF82C64012030710421DFF82804FFF794FA002030707070B07020682843206001
:2037C000206820F440502060DFF80C04082101700020BDE87040FEF757BB10B5DFF8EC4375
:2037E0002068800703D5206820F0020020602068800606D52068400403D5206820F0200083
:020000040800F2
:2038000020602068C00506D500F04FF818B9206820F4807020602068400606D5FFF78DF8C8
:2038200018B9206820F0400020602068400506D500F016F918B9206820F480602060206863
:2038400000050ED500F00CF938B14FF40041DFF88C03FFF735FA012803D1206820F400609A
:203860002060206880050AD54FF48051DFF86403FFF726FA18B1206820F400702060206897
:20388000400703D5206820F0040020602068000703D5206820F008002060206840F67E71B9
:2038A0000140481E8041C00F10BDF0B4CC490868C0EB8010CB4A128910188009CA4A1268B1
:2038C0004FF416739A4238BF47F230500860BA48C64A1278032A0CBF028AC2898281096849
:2038E00045F2E95245F6D523994209D3C04CB4F900408589261204EBD65405EB642409E0B3
:20390000914206D384895D1A0326B5FBF6F5641B00E00024048191423CBFB649012203D3E5
:20392000994202D3B34900220A70B349096840F2E93240F2D173994209D3AD4CB4F9004072
:203940008589261204EBD65405EB642407E0914223BF8489C1F5FA65A4EB950400244481C1
:2039600091423CBFA549012203D3994202D3A34900220A7041890289914228BF1146A04A0A
:2039800012885201A2F5F075ADB29E4A1278012A23D19D4A1268AA421FD283889B4C247882
:2039A0009B4E3678ED1A05F240157543A71B95FBF7F5ADB2A3F5A07797420BD26C4394FB25
:2039C000F6F4A4B2D21AAA1802F240125143B1FBF4F102E0714391FBF4F1C1800020F0BC7A
:2039E0007047F0B47F4C7448C169226811EB5242C261016AA38859180162238A456A5D1942
:203A0000866AA489A6190478671C4478FFB2FE2F0ED18032120A403A82617B4D2A6006F1DE
:203A20008002120A744D2A600027C76100253E46077086624562774A1568C5EB05255B1913
:203A40001B0A1360621CD2B2082A06D1091DC9085D4A11600021016200224270F0BC7047F9
:203A600010B56D48B0F90000674909685F4A1278032A12BF01EB400000EB400301EB430048
:203A8000664908600CBF6648664800884A4CA080608AA28A096843F61913994208D30020E8
:203AA0004FF496718A4226BF0121A170521C1BE0A28891420ED200224FF4C871884238BF33
:203AC000401C11D30221A17057490B8843F004030B8009E002F28430884224BF00200022FA
:203AE00002D200200022A070A28260824FF400413A48FFF7E5F8012804BF0020A07002D0D3
:203B0000A078022805D0484908884FF6FB7210400880A07810BD2848806900B270474348B1
:203B200000218161424881614248816142488161704710B5264C2078401C2449096840F648
:203B40007E7211422070C0B222D03C2832D300202070A078E178884201D2207928B9042168
:203B60001C48FFF7BAF8012007E004211948FFF7B2F80020A178491CA17020716078401C97
:203B80006070C0B2142815D300206070A07010BDC8280FD300202070607980F00101617153
:203BA0000C4821B10421BDE81040FFF794B80421FFF793F810BD0000B40000209400002088
:203BC00096000020002C0140CC030020BC030020A0030020000C014068040020000801400F
:203BE000F803002038000020C00300205F0100203404002080040020D40300208104002057
:020000040800F2
:203C00005201002061010020C40300206001002062010020D00300209A00002008040020EB
:203C20004C0100204A0400204E0100201C030020F8020020D40200206000002070477047FD
:203C40001648B0F90800704714480121417000210170018141818180C180704780B54FF428
:203C60008070ADF8000028208DF8030000A90C48FEF7BDFF4FF40040ADF8000004208DF860
:203C8000030000A90748FEF7B2FF07480021016001BD0648002101807047000038010020F4
:203CA000000C014000080140C0030020200400202DE9F74F84B09946DFF8E843B4F90E809B
:203CC00047F6FF7101FB08F0E26A9042B8BFE06207DB4FEAC8335B429342A4BFA8EBC832F4
:203CE000E262226B904206DB4FEAC8304042904202DBA8EBC8302063B4F90C004143626AC7
:203D00009142B8BF616206DBC3035B429342A4BFA0EBC0326262A26A914205DBC1034942CB
:203D2000914202DBA0EBC031A162656A95FBF0F6BDF81810711A0FB2A16A91FBF0FBBDF8AF
:203D40001A00ABEB000000B20190B4F908C004980FFA89FE0EFB00F9E16A91FBF8F0B4F961
:203D60001420B4F91630B4F912A036B206FB1A5507FB0C554FEAA93609EB5646760036149A
:203D800006FB035500B200FB12550395B4F9105005FB08F50095C44DB5F90050B4F918604B
:203DA0006E43D4F83090B4F90AC007FB0C1C009F99FBF7F707FB06C70297B4F908C0059F83
:203DC0000EFB07FE99FBF8F8A76A0FFA8BFB0BFB1A77DDF804A00AFB0C7C4FEAAE370EEBFD
:203DE00057477F003F1407FB03C30FFA88F808FB1237B4F90A200AFB0292009B91FBF3F13B
:203E000001FB1626A949B1F9001021B1002D48BF4FF0FF3200D40122A080A4F8068002FB12
:203E200008F1494209B2504300B200F0D6F8B4F920100A4602F1500383420EDA9C4BB3F98D
:203E4000003040F22D15AB4205DA9A4B1B889A4D2D68AB4201D201F1500000B2503A9042DE
:203E60000EDA934AB2F9002040F22D139A4205DA904A1288904B1B689A4201D2A1F1500022
:203E80008C4909888C4A126891420CD28B490978012904D08A49B1F90010D32903DB00B24F
:203EA0001428B8BF142087490880B1F900502584284600F0D7F88448018869180180039801
:203EC00060620298E062A7622663804800684FF41671884239BF40F2891040F25E7140F2F8
:203EE0004D2040F6D701E182608207B0BDE8F08F70B4002200217648034610245D5EB3F91E
:203F000002607519B3F904607519B3F906607519AA180833641EF1D1531102EB9362921149
:203F2000614B1A80102330F9024BA41A04FB041130F9024BA41A04FB041130F9024BA41A44
:203F400004FB041130F9024BA41A04FB04115B1EE9D15448931102EB5362D211C38B5A4322
:203F60004B1101EB9361B2EBA11FB4BF00210121817070BC70474B48807870474A4800E06A
:203F80005148B0F9000070474648002141628162C162016381704163017041704A480180A2
:203FA0006DE0404902884A8242880A8182888A82C2884A810289CA8242890A8382898A8110
:203FC000C289CA81028A0A82428A4A83828A8A8382698A63808BC8837047F8B504460D4652
:203FE0003948B0F9000002F0EFF90090BDF9020000FB04F2BDF9001001FB05F3354E9F1890
:020000040800F2
:204000007780684301FB04003080981303EB5040C11309B2901302EB504040000014BDE87D
:20402000F440204AB2F91A30081A5843516B431300EB93404B1401EB9331891401EBA030F8
:20404000916B814203DA01201070084608E049428842BCBF01205070F7DB00211170517007
:2040600000B270471C490A78521CD2B2402A08BF00220A700978164A22F81100704700B5B9
:204080008021134802F02AFB13480021017000BD0448B0F9040070470248B0F90600704703
:2040A00000000000640200203C0400209C000020360400202C040020DC0300207B04002016
:2040C000380400203E0400203A040020F4030020640100201404002089040020704750F844
:2040E000041B61B150F8042BD30744BFA9F101039A18002342F8043B091FFAD1EFE77047CF
:2041000000B589B040F28910ADF8000040F24F20ADF8040040F25E70ADF808000120ADF884
:20412000100040F2FA3000EBD070C0030014BDF810104900ADF810100028F4D109044811DB
:2041400002F0D0FA384A394B02F0E4FA0022384B02F0E0FA02F0B0FBADF80A003548ADF8EE
:20416000020041F6F450ADF8060040F66410ADF8120040F2A910ADF814004FF48040ADF86A
:204180000C004FF48060ADF80E0041F2257006900820ADF81C0000A8FFF703FF09B000BDE0
:2041A00080B5FFF7E8FE50B923480178491C0170C9B232290AD300210170002002BD00F017
:2041C00007F81028F0DB1C4800210170012002BD80B5FFF7D3FE1A4948434FF47021FFE763
:2041E00090FBF1F000B202BD1448017801B1704780B5417081704FF42021C1601149B1F924
:2042000000100121017000F004F80F480421017001BD0A48002101708160C16081800B482A
:204220000521018070470000A7E8482EFF2109400000F03E00B0FFFF880400208003002087
:20424000007102001E040020680400208402002010B586B025208DF8040001208DF8050003
:2042600000208DF8060001208DF8070001A8FFF7D0F901214FF48040FEF736FC01210920E7
:20428000FEF732FC01210420FEF731FD4020ADF8000003208DF8020018208DF80300DFF84C
:2042A0000C4700A92046FEF7A2FC8020ADF8000004208DF8030000A92046FEF798FC4FF43D
:2042C0001650029000200390ADF81000ADF814000C20ADF81200DFF8D84602A9204602F0EA
:2042E00017FB012240F22551204602F067FB002240F22771204602F061FB0121204602F00D
:2043000053FB06B010BD38B5DFF8A8060578DFF8A846032D40D32078462815D16078582891
:2043200012D1A0780C280FD1E078FF280CD1DFF88C0600210180DFF8880601880C2980F074
:204340003383C91C018031BDA91E204601F0A8FA291911F8022C11F8011C01EB022189B2AA
:204360008842E4D12078462816D16078432817D1DFF85006DFF8281D09680160DFF8240D83
:2043800001884FF6EF7211400180DFF83406018851B1491E018007E02078462840F0F88201
:2043A0006078432840F08380A078112810D1E078012800F0F982112820D12079002840F04E
:2043C00089806079002840F08580112111201FE0162840F07F80E07811281CD12079002890
:2043E00078D16079022875D1A079DFF8201D0870E079DFF81C1D08701621E7E712283BD15A
:020000040800F2
:204400002079002866D16079002863D111211220BDE83440E4E2122815D12079002859D121
:204420006079012856D1A079F12804BFDFF8600D012104D0F02803D1DFF8540D002101706E
:2044400016211220E4E7132844D12079002841D1607901283ED1A079002803BF0021DFF8F9
:20446000682511800121DFF8702D1070DFF85C05017016211320CBE7142806D1207948BB94
:20448000607938BB11211420C2E7182806D1207900BB6079F0B911211820B9E7202819D118
:2044A0002079B8B96079A8B911212020B0E7422810D1A078112810D1E078402810D12079F8
:2044C000002840F071826079002840F06D82112140209DE7607842281ED1A07811282ED1DA
:2044E000E078412806D1207948BB607938BB112141208DE7422806D1207900BB6079F0B99E
:204500001121422084E7442819D12079B8B96079A8B9112144207BE7432810D1A07811286D
:2045200011D1E07861283BD12079002840F03C826079002840F038821121612068E7607838
:20454000432840F0A081A078162827D1E078612832D12079002840F0AC81A079F1280BD141
:20456000DFF8940D01210170DFF8900DF1210170DFF88C0D00210DE0F0280CD1DFF8780D6A
:2045800000210170DFF848040068302803D2DFF86C0DF02101701621612039E7112870D1AD
:2045A000E07863282ED1207900286AD16079002867D1112163202BE7632840D120790028C0
:2045C00040F077816079012840F07381A079F1280FD14FF40041DFF82C0DFEF771FB70B95D
:2045E000DFF8EC030068302809D2DFF8140D012104E0F02803D1DFF8080D002101701621BB
:20460000632005E7712808D12079002839D16079002836D111217120FAE6722806D1207939
:2046200078BB607968BB11217220F1E6802828D1207930BB607920BB11218020E8E681288E
:2046400033D12079002840F034816079032840F03081E079000611D5207A78B9DFF8BC0D1B
:2046600001884FF67E7211400180DFF86803016821F010010160002002F08BFC162181200B
:20468000C6E6A07811280DD1E078822831D12079002840F00E816079002840F00A811121CD
:2046A0008220B5E6162840F0B280E07890283AD12079002840F0AB806079042840F0A7808A
:2046C000A079012812D1207AA0F11E01C9B207290CD2DFF8881D00EB8002607A00EB4000F4
:2046E00000EB82100880BC4809880180162190208EE690280AD12079002840F0DA8060798D
:20470000002840F0D6801121902081E691282CD12079002840F0CD806079002840F0C98034
:204720001121912074E691282CD1207900286ED1607902286BD1A079E17901EB002080B296
:20474000322838BF322002D3B52828BFB420DFF8941D152250430A2290FBF2F008809F48EF
:20476000098801801621912052E6922839D12079002840F09E806079002840F09A801121B7
:20478000922045E6922842D1207900283FD1607904283CD1A079DFF8501D0870E079217AC3
:2047A00001EB0020DFF8B41C0988490980B2884238BF0846DFF8341D0880607A032838BF76
:2047C000032002D3152828BF1420DFF844190978884228BF481EDFF8181D08701621922050
:2047E00016E6A02808D12079002862D1607900285FD11121A0200BE6B0281DD1207900288D
:020000040800F2
:2048000057D16079002854D11121B02000E6A07816284ED1E078B1284BD12079002848D1C6
:204820006079042845D1A079E17901EB002080B20A280AD20A200BE0B1283AD12079C0BB91
:204840006079B0BB1121B120E2E5B52828BFB420152148430A2190FBF1F0DFF8981C088047
:20486000207AA0F11E01C9B2072909D200EB8001607A00EB400000EB8110DFF87C1C088084
:204880001621B120C4E5582813D1A0780C2840F08B80E078E02840F087802079002840F0F4
:2048A00083806079022840F07F80DFF8500CFA2179E06078432877D1A07811280BD1E0780C
:2048C000F12821D1207900286ED1607900286BD11121F1209CE5162866D1E078F12829D1EC
:2048E0002079002860D1607902285DD1A079E17901EB0020411E89B2B1F5616F3CBFDFF834
:20490000001C08801621E4E7F22808D1207900284AD16079002847D11121F22078E5F3284D
:2049200042D1207900283FD1607900283CD11121F3206DE5F32813D12079002834D1607950
:20494000022831D1A079E17901EB0020411E89B2B1F5616F3CBFDFF8AC1B08801621E7E776
:20496000212821D1207900281ED1607903281BD1A079552818D1E079502815D1207A442820
:2049800012D11348006830280ED2162121203FE55A2809D1A078532806D1E078312803D152
:2049A000DFF8640B0121017031BD0000000C0140003801406A040020E40100205601002060
:2049C0005C040020E40300203204002078040020E0030020BC0300204A040020C20000202C
:2049E0002DE9F04387B006460F46DFF8B40600680528C0F02B81DFF8144BDFF8145B2878F8
:204A00002178884205D202F090FB287821788842F9D3FF2E40F01D81DFF8F86A46203070D6
:204A200058207070B770FF20F07000203071222070711120B071DFF8E07A386800EB800006
:204A4000C008DFF8D819098821B1DFF8BC1A097801B900200104090EF171307240207072F9
:204A6000DFF8B80AB0F90000024615215528A6BF1B324FF4FA734FF425735A4392FBF1F1B0
:204A80006FF0F90209B29142BEBF4942DFF8902A114302DB002948BF002109B20A12B27218
:204AA000F17241213173DFF8E01DB1F90020DFF8DC1D0968DFF854361B78032B06D0032390
:204AC00092FBF3F39A185218A12302E001EB8202A3235A43D20980B20A2802D2A12048436F
:204AE000C209DFF8400A018841F6417399420DD30B4692B203F1640E9645B8BF01F16402F6
:204B000004DB643B9A42B8BFA1F16402028092B2100A7073B2734220F07300F005FD01022A
:204B20004FF47A7291FBF2F189B20A0A327471744421B1744FF00A08401D90FBF8F0F074EE
:204B40005221317570754FF40041DFF8B807FEF7B7F8012818BF002003D1707D022801D2BB
:204B6000022070756120B075DFF890070178F175DFF83095B9F80010DFF87C271278012AAF
:204B800005D1F122F2754FF6FD72114005E03A681AB9F022F27541F00201A9F80010F17D9A
:204BA00001708020307600F095FE01127176B0767220F076DFF8D80C018808FB01F14FF427
:204BC0008E72B1FBF2F2DFF8CC1C0B8808FB03F340F22B17B3FBF7F317043F0E37777277EF
:204BE0001A04120EB277F377002202800A80822086F82000DFF8A00C0068010E86F82110CD
:020000040800F2
:204C0000010C86F82210010A86F8231086F82400E02086F82500B9F80000010A86F8261066
:204C200086F827002821304600F03AFE011286F8281086F829002A202070002028700122C3
:204C400040F22771DFF8540C01F0B8FE07B0BDE8F083E02E20D1DFF8BC6846203070582065
:204C60007070B770E020F0700020307102207071DFF830040788380AB071F7710821304605
:204C800000F00EFE0112317270720A20207000202870002FDAD0D2E7012E1DD1DFF87468AC
:204CA00046203070432070701120B0700120F07000203071052070715220B0714520F071B9
:204CC00041203072442070725920B072B220F0722C2030730D20AFE7112E1DD1DFF834686A
:204CE0004620307043207070B7701120F0700020307102207071DFF814040078B071DFF890
:204D000010040078F0710821304600F0C9FD0112317270720A208FE7122E1DD1DFF8F467B9
:204D20004620307043207070B7701220F0700020307101207071DFF85804007801280CBF0F
:204D4000F120F020B0710721304600F0A9FD0112F171307209206FE7132E19D1DFF8B4672A
:204D60004620307043207070B7701320F0700020307101207071DFF860040078B071072171
:204D8000304600F08DFD0112F1713072092053E7142E21D1DFF87C67462030704320707072
:204DA000B7701420F070002030711820707100A80FF66451B1E88C51A0E88C51182200A93E
:204DC000B01D02F0C3F91E21304600F069FD0112B177F07720202FE7182E21D1DFF83467AB
:204DE0004620307043207070B7701820F070002030711820707100A80FF63451B1E88C5129
:204E0000A0E88C51182200A9B01D02F09FF91E21304600F045FD0112B177F07720200BE738
:204E2000202E1BD1DFF8EC664620307043207070B7702020F07000203071182070711822EB
:204E4000DFF8581CB01D02F081F91E21304600F027FD0112B177F0772020EDE6402E39D1D8
:204E6000DFF8B0664620307042207070B7704020F0700020307102207071DFF8A006B0F92C
:204E80000000024615215528A2BF02F11B004FF4FA725043BCBF4FF42570504390FBF1F014
:204EA0006FF0F90100B28842BEBF4042DFF87016084302DB002848BF002000B20112B17163
:204EC000F0710821304600F0EBFC0112317270720A20B1E6412E38D1DFF8386646203070AF
:204EE00042207070B7704120F0700020307102207071DFF89409B0F90020DFF890090168AE
:204F0000A320824B1B78032B05D0032392FBF3F39A18521801E001EB82024243D209DFF82E
:204F2000FC35B3F900309BB20A2B3CBF4843C2091004000EB071F2710821304600F0B0FCB0
:204F40000112317270720A2076E6422E20D1DFF8C4654620307042207070B770F0700020E3
:204F600030710220707100F0DFFABC2148434FF47A7190FBF1F080B2010AB171F0710821D9
:204F8000304600F08DFC0112317270720A2053E6442E1CD1DFF87C654620307042207070C8
:204FA000B7704420F070002030710120707100F0BBFA401D0A2190FBF1F0B07107213046EB
:204FC00000F06EFC0112F1713072092034E6612E18D1DFF840654620307043207070B770B9
:204FE0006120F0700020307101207071C3480078B0710721304600F053FC0112F171307275
:020000040800F2
:20500000092019E6632E1DD1DFF808654620307043207070B7706320F07000203071012070
:205020007071B74890F9000001280CBFF120F020B0710721304600F033FC0112F1713072FD
:205040000920F9E5712E2FD1DFF8C8644620307043207070B7707120F0700020307108205D
:205060007071DFF83C0A0088010AB171F071DFF8340A0088010A31727072DFF82C0A00687A
:20508000010EB172010CF172010A317370730E21304600F005FC0112B173F0731020CBE5CC
:2050A000C00300204E010020722E33D1DFF864644620307043207070B7707220F0700020D9
:2050C0003071042070710A22DFF8E009006850434FF48E71B0FBF1F0DFF8D41909685143AC
:2050E00040F22B12B1FBF2F10204120EB271F0710804000E307271720A21304600F0D0FB0D
:205100000112B172F0720C2096E500BF5F01002060010020802E1AD1DFF8F86346203070BF
:2051200043207070B7708020F070002030710220707100F0CFFB0112B171F0710821304652
:2051400000F0AEFB0112317270720A2074E5812E20D1DFF8C0634620307043207070B77091
:205160008120F0700020307103207071DFF844098179B171C079F07100203072092130462D
:2051800000F08EFB01127172B0720B2054E500BF76040020822E21D1DE4E4620307043208A
:2051A0007070B7708220F0700020307104207071DFF8E4060068010EB171010CF171010A4C
:2051C000317270720A21304600F06AFB0112B172F0720C2030E500BF79040020902E26D16A
:2051E000CC4E4620307043207070B7709020F07000203071042070710120B0710020F0718C
:20520000964800884FF4A07190FBF1F23272327A01FB1200032190FBF1F070720A213046F5
:2052200000F03EFB0112B172F0720C2004E5912E20D1B84E4620307043207070B7709120C1
:20524000F0700020307102207071A648008800EB80014800152190FBF1F080B2010AB171FF
:20526000F0710821304600F01BFB0112317270720A20E1E4922E1FD1A64E46203070432094
:205280007070B7709220F070002030710420707195480078B07195480088010AF171307245
:2052A0009348007870720A21304600F0F9FA0112B172F0720C20BFE4A02E25D1954E4620C1
:2052C000307043207070B770A020F0700020307102207071DFF8E0070078B071DFF8DC07CF
:2052E0000078F0710821304600F0DAFA0112317270720A20A0E400BF77040020820400202C
:205300006E04002000080140B02E19D1814E4620307043207070B770B020F07000203071BA
:20532000022070710020B07100F06EFBF0710821304600F0B5FA0112317270720A207BE410
:20534000B12E2ED1734E4620307043207070B770B120F07000203071042070716548008812
:2053600000EB80014800152190FBF1F080B2010AB171F071604800884FF4A07190FBF1F225
:205380003272327A01FB1200032190FBF1F070720A21304600F084FA0112B172F0720C206A
:2053A0004AE4F12E19D15B4E4620307043207070B770F120F07000203071022070715048D0
:2053C0000088010AB171F0710821304600F068FA0112317270720A202EE4F22E20D14D4E46
:2053E0004620307043207070B770F220F0700020307104207071DFF8C8060068010EB171C7
:020000040800F2
:20540000010CF171010A317270720A21304600F047FA0112B172F0720C200DE42A040020B8
:20542000F32E1DD13B4E4620307043207070B770F320F0700020307102207071314800882C
:20544000010AB171F0710821304600F029FA0112317270720A20FFF7EFBB00BFB800002013
:20546000212E7FF4F3AB2B4E4620307043207070B7702120F0700020307107207071062053
:20548000B0715220F07145203072422070724F20B072F072542030730D21304600F000FA35
:2054A00001127173B0730F20207000202870012240F22771DFF8E40301F080FA207829780C
:2054C0008142FDD3012080F31388DFF8F805016801F4E061DFF8F02511430160BFF34F8F66
:2054E000FEE70000C0000020610100205201002062010020C40000204C010020630100209A
:205500004A010020540100207B040020750400206B040020A0020020E003002038040020C3
:205520000080FFFF66040020F8B5D8480068DFF89C4521686539B1F5F97F0BD9D249B1F988
:205540000010DFF88C251278032A14BF00EB410000EB81004FF4A075DFF878150988A03173
:2055600091FBF5F1C9B2222908BF462212D0232908BF1E220ED0242908BF11220AD0252942
:2055800008BF0A2206D0262908BF062202D0032222290DDBC0F54D5101EB81035900B1FB12
:2055A000F2F101F525514FF425525043B0FBF1F0DFF82465F0603069B0F5165F21D9F1680D
:2055C00088420CD24FF40041DFF81005FDF778FB0128306906D1318921B9401C02E081421E
:2055E00001D2401EF0603089401C3081A649B1F90010C911C1F1040180B28142BCBF00209A
:205600003081F0683061DFF8D4744FF400413846FDF756FB0128F06840F08280B0F5275FAC
:2056200001D200251FE0B0F52C5F1ED2A0F5275096214843B0FBF5F540F2B630ADB2854232
:205640000BD370694821B0FBF1F101F2B632954238BF01F2B635401C706140F2B630ADB272
:20566000854280F0B7800020C8E0B0F5315F08D2A0F52C5096214843B0FBF5F000F1960576
:20568000DAE7B0F5365F08D2A0F5315096214843B0FBF5F000F22C15CEE7B0F53B5F08D24C
:2056A000A0F5365096214843B0FBF5F000F5E175C2E7B0F5405F09D2A0F53B5000EB80015E
:2056C0004801B0FBF5F000F25825B5E7B0F5455F09D2A0F5405000EB80014801B0FBF5F058
:2056E00000F2F825A8E7B0F54A5F08D2A0F5455032214843B0FBF5F000F298359CE743F2D5
:205700006041884209D2A0F54A5000EB80014800B0FBF5F000F2CA358EE740F2DE3590E7AE
:20572000B0F5255FFFF47DAFB0F52A5F06D2A0F5255096214843B0FBF5F58EE7B0F52F5F92
:2057400008D2A0F52A5096214843B0FBF5F000F1960582E7B0F5345F08D2A0F52F509621BC
:205760004843B0FBF5F000F22C1576E7B0F5395F08D2A0F5345096214843B0FBF5F000F587
:20578000E1756AE7B0F53E5F09D2A0F5395000EB80014801B0FBF5F000F258255DE7B0F58A
:2057A000435F09D2A0F53E5000EB80014801B0FBF5F000F2F82550E7B0F5485F08D2A0F503
:2057C000435064214843B0FBF5F000F2983544E740F2E73520684FF47A71884209D330785A
:2057E00001280CD04FF400413846FDF769FA012805D1A5F2B63000EBC001C80070614FF447
:020000040800F2
:2058000000413846FDF75CFA30704FF47A70854228BF40F2E735F088012803D1B580758017
:205820000020F0804FF400413846FDF749FA012809D17088854238BF0546284629460A2D87
:2058400011D20A250FE0B0880146A84205D201F22C118D4205DA054603E0481B0830A1EBD4
:20586000201529462846B1809D490968090504D50025002042F6E011316170809948058051
:20588000A8B2F2BD000000009A000020C40300204C0400204E0400200404002000380140DB
:2058A00030B4002299B141F22103491E10F8014B82EA042292B208245500120446BF83EAA7
:2058C000050292B2AAB2641EF6D10029EDD1104630BC704738B5844C2078000606D5802022
:2058E000208004218148FDF7F8F901E0002020807A48FDF7E7F97A4D29682088890502D49A
:205900002968C90601D540F001002968090504D54FF6FB71084040F002002968490504D5C5
:205920004FF6FD71084040F004002968090748BF40F008002968890648BF40F040006C490C
:2059400009684FF21962914228BF40F0400020802868C00611D55D4800684FF41671884273
:205960000BD22178090608D4332806D3802001F010FB208840F08000208020885D4909782F
:2059800001290BD04A490968A1F6B8314CF2BC52914203D258490978012902D14FF40071B7
:2059A0000843296849060ED45449096840F6B83289B2914207D352490978282906D24349F3
:2059C0000968C92902D34FF4807108434D490988C82251433D4A12684B4B1B68D21A914292
:2059E00003D34A4A1288914201DA40F400604849097809B140F400504649097809B140F413
:205A000080402080208832BD30B439490A684FF249118A4228BF6FF0270335D201200FF2B7
:205A200028118C1C34F8025B954211D201EB400333F8023C0A2404FB00F5323D9A1A6243C0
:205A400031F81010591AB2FBF1F14B191BB21BE0401C34F8025B954222BF401C34F8025B4D
:205A6000954222BF401C34F8025B9542DED3401C34F8025B9542D9D3401C34F8025B9542DD
:205A8000D4D3401C1928CDDBC0B2182828BFC82303F13200C0B230BC7047000064030020D4
:205AA0002204002024040020E803002000040020CC030020E40100207C0400207D040020F4
:205AC000FC0300200CED00E00400FA05C00300205F010020B8000020FC000020000801402B
:205AE000BC030020460400202A040020000C0140D40300206F040020870400203800002035
:205B00007304002044040020E40300205E0400208004002081040020535F4543555F5A5F0D
:205B200046575F4C535F56332E305F312E392E34535F4543555F5A5F48575F4C535F5633FF
:205B40002E305F312E302E3448F1B4E897DCB1CC15B93EA3A28B7D74FE5EB74B943C052FA3
:205B6000A224A51C6C16DC11090E060BE5083707E105C60408046F03EE02000070B582B067
:205B8000DFF83845002020806080DFF83405002101804180DFF82C0501804180DFF8285500
:205BA000DFF82865DFF82825705E01F065FB2860DFF82025B4F90210B6F9020001F05CFBE2
:205BC000686000F0B8FBD5E9001200A800F0D3FBDFF80425DDE90001C2E90001D2E90001F5
:205BE00002B0BDE87040FBF7CFBEF0B585B0FBF77BFE0090DFF8C80400A90A8802804A8818
:020000040800F2
:205C0000428002880A8042884A80009800F00EFB0190DFF8B05401A8018829804188698090
:205C2000FEF7AEF900A92A880A806A884A800146009800F019FB0190DFF8806401A80188C6
:205C4000318041887180DFF8940431880180FEF74FF9FDF760FF0346DFF87C4400A8298867
:205C6000018069884180009AD4E90001FEF720F8DFF86C04B0F9000068B9DFF86804B0F98F
:205C80000000332807DBDFF860040078012808BF6FF0090000D00020DFF83074A7F846006C
:205CA000B6F90010DFF82824DFF840040068400406D4B7F84000B7F84630181800B203E088
:205CC000DFF82C04B0F9000001F0D6FADFF8F8532860DFF80024B6F90210B7F9020001F04A
:205CE000CBFA0128A8BF00206860FEF7D1F9B862FEF7D2F9F862FEF741F9A7F84400332807
:205D00001BDBB7F84A10491C09B2C92903DBC921012287F83020B7F9482064280FDAB7F97B
:205D2000400060B9501C40F2F51200B2904207DB0020002187F8301002E00021EBE700200A
:205D4000A7F84800A7F84A1000F0F5FAD5E9001202A800F010FBDDE90201C4E90001D4E9DB
:205D60000001FBF711FEFCF7B9FD05B0F0BD10B582B0FEF72DFADFF87C43DFF87C230146B0
:205D8000DFF87803B0F9000001F076FA20800020608000A82188018061884180CB4800A9CF
:205DA0000A8802804A884280D54902880A804088D449088002B010BDC448D14909880180E5
:205DC000D049098841807047C04842F6E06181804021C1804FF4007101814FF400614181E1
:205DE000C949C16000210161C168C902416100218161C16101844FF40041418400214162A0
:205E0000C249B1F90010018700218187704770B5AE4C221DB4F93E10B4F93A0001F02CFAFE
:205E2000A087B4F84200A18F0818B54909880818A4F84000B6480078401E0501ADB2B5483C
:205E4000008840F29111884213D3B34E306885420FD2FEF793F833280BDB3068281A9621A3
:205E60004843A3490880AD4A00B29042B8BF0A8004DB9F48B0F90000002807D59C49B1F9A5
:205E80000000B4F94010814207DA04E0B4F94000002802D50020A4F8400070BDA04820213F
:205EA000018001214180002181800121C180002181830121C183002101629349816000220B
:205EC000C2600161426182618048A0F8422070472DE9F04F81B040F21E30924C20808C4DE2
:205EE00029784FF00F0801EB410252000A2392FBF3F208FB01228A4FBB69744E96F832C026
:205F00000B290DD392B202FB02F14FF4887291FBF2F213F57A7FACBF002303F2E83301E00C
:205F20000121B980BB6180490A800CF10102D2B2072A28BF002286F83220B6F84C2096F861
:205F400032303BB909888A4238BF521C02D3914238BF521EA6F84C2041F24A09B6F84C1080
:205F600009FB01F191FBF0FAFEF708F86F494843C11300EB1140001448BF4042DFF864B1E4
:205F8000ABF8000096F8330029780B2938BF642108D36749098891FBF8F13D31C9B2472962
:205FA00028BF4621401CC0B2062828BF002086F8330096F8340096F8332032B9884238BF90
:205FC000401C02D3814238BF401E86F8340096F834106420574A1288574B1B689A422FBF46
:205FE00089033F4AB2F90020514391FBF0F044F2010100B28842A8BF4FF480400FFA8AF11F
:020000040800F2
:2060000048433A46BBF90010431300EB93408000001401F031F9A6F84200BBF90000716D7C
:206020004118716596F83520521C86F83520D2B2102A06D1083109093165002186F83510B3
:20604000716596F831104B1C86F831303B490A68DBB2642B2DD3002386F83130336D2488F5
:20606000241F634393FBF9F31C463C28BCBF012086F8360009DB6528A4BF002086F83600FF
:2060800004DA96F83600012800D10024224804609A18B2F5345F0CD929480078012808D1B6
:2060A0000022284803685B1C0360274803885B1C03800A6001B0BDE8F08F0000B8030020FB
:2060C000B0030020B4030020900300205C000020F8020020D40200209803002034040020C4
:2060E00040040020360400207F040020BC03002042040020AC0300201C0300201E040020AA
:206100001C0400201A040020D9B1FFFFBA0000206001002050040020E00300206CEEFFFF4F
:2061200040030020440100204601002000710200480400202C040020DC030020F0030020EF
:2061400077040020E803002024040020324847F6FF4141603149F0220A7000218160072189
:20616000016070472E49888070472D488188FFE7481E8041C00F704729494000488070478F
:2061800027498881704726488189F1E738B5244CA08908B1401EA081A08810B1A088401E52
:2061A000A080E08810B1E088401EE080208910B12089401E2081608808B1401E6080608996
:2061C00010B1401E60810EE001206081154D2878032808BFFDF782FF2878042803D1FDF7D2
:2061E0007DFFFDF7DDFF207818B12078401E207031BD012020700B4D0B480068C007287853
:2062000005D5042807D1BDE83140FFF7B0BD042808BFFFF7D1FD31BD10E000E023ED00E0C2
:206220002801002068040020BC03002001B481B0BDF90400ADF8000044F6E610BDF904106B
:206240004143BDF9062050438A1301EB5241C9134942821300EB5240C013A1EB4000ADF872
:206260000200009802B0704771B481B0A1F500400004800D4FF44071014012D0B1F5807FA2
:2062800006D0B1F5007F21D0B1F5407F16D027E00FF24821C0F1FF02D2B231F91220524230
:2062A0001BE00FF23821C2B231F912205242C0F1FF00C0B231F91000434211E00FF21C2115
:2062C000C0F1FF02D2B231F91220F2E70FF20C21C2B231F91220C0F1FF00C0B231F91030C9
:2062E00036490B804A80B1F90000BDF9042000FB02F3B1F90210BDF9064001FB04F59E13F8
:2063000003EB5643DB13AE1305EB5645A3EBE533ADF80030514360438A1301EB5241821359
:2063200000EB5240C01300EBE130ADF80200009802B070BC704710B421484168026801FB01
:2063400001F302FB02331F4CA34212D31B0E3E3BDBB20FF2041434F813305A43941302EBFA
:206360005442D213026059438A1301EB5241C913416010BC7047F0B5104EB6F9003003FBA8
:2063800001F7B6F9026006FB02F4BD1307EB55474FEAA43E04EB5E44E41304EBE73771433B
:2063A0005A438B1301EB5341C9134942931302EB534201EBE231C0E90071F0BDA803002002
:2063C00090030020D2A6B83E81B0A0F500400004800D4FF44071014021D0B1F5807F29D041
:2063E000B1F5007F03D0B1F5407F0AD031E00FF2EC01C2B231F81220ADF80220C0F1FF0021
:020000040800F2
:2064000022E00FF2D801C0F1FF02D2B231F81220ADF80220C0B231F91000404217E00FF222
:20642000BC01C2B231F912205242ADF80220C0F1FF00EFE70FF2A401C0F1FF02D2B231F9E8
:2064400012205242ADF80220C0B231F91000ADF80000009801B070477B7F777E797D817C7C
:206460008F7BA27ABA79D778FA7721774C767C75B074E8738673C47206724B719470E16F82
:20648000306F836EDA6D336D8F6CEE6B4F6BB46A1B6A8469F0685E68CF674267B7662F6638
:2064A000A8652465A1642164E1636463E8626E62F6617F610A6197602560B55F475FD95E88
:2064C0006E5E035E9B5D335DCD5C685C045CA25B415BE15A825A255AC8596D590000C900DB
:2064E00092015B022403ED03B6047F0548061107D907A2086A09330AFB0AC40B8C0C540DEA
:206500001C0EE30EAB0F72103A110112C8128F1355141C15E215A8166E173318F918BE1943
:20652000821A471B0B1CCF1C931D571E1A1FDD1F9F2061212322E522A62367242825E825B6
:20654000A82667272628E528A329612A1F2BDC2B992C552D112ECC2E872F4130FB30B53124
:206560006E322633DF3396344D350436BA366F372438D9388C39403AF23AA53B563C073D66
:20658000B83D683E173FC53F73402141CE417A422543D0437A442445CD4575461C47C3474A
:2065A00069480F49B449584AFB4A9D4B3F4CE04C814D204EBF4E5D4FFB4F97503351CE5186
:2065C000685202539B533254C9546055F5558A561D57B0574258D3586459F359825A0F5BAD
:2065E0009C5B285CB35C3E5DC75D4F5ED75E5D5FE35F6860EB606E61F0617162F162706346
:20660000EE636C64E8646365DD655666CF664667BC673268A66819698B69FD696D6ADC6AA1
:206620004A6BB76B236C8E6CF86C616DC96D306E966EFB6E5E6FC16F22708370E270407102
:206640009D71F9715472AE7207735E73B5730A745F74B27404755575A575F37541768D7673
:20666000D87622776B77B377FA773F788478C77809794A798979C879057A417A7C7AB67ADC
:20668000EE7A267B5C7B917BC57BF87B297C597C887CB67CE37C0E7D397D627D897DB07DF9
:2066A000D57DFA7D1D7E3E7E5F7E7E7E9C7EB97ED57EEF7E097F217F377F4D7F617F747F53
:2066C000867F977FA67FB47FC17FCD7FD87FE17FE97FF07FF57FF97FFD7FFE7F002200F036
:2066E00003BE0000010040F10880F446404200F004F851F000416047010009D0B0FA80F159
:206700008840C91CC1F58461090501EBD021400570470000B0B581EA030C0CF0004C40F2F1
:20672000FF7515EA11541DBF15EA1357AC42AF4239E0E41923EA455343F48013C90241F0DC
:20674000004141EA505EC7021100A7FB020200284FF00000EEFB01204FF00001E3FB0721E8
:2067600018BF42F00102401800214941E3FB0E01A4F580640F0302D252004041494154F118
:2067800001046CDD470872F1004250F1000051EB0451A1F580115CBF41EA0C01B0BD4CEAC8
:2067A00005510020B0BD05EA1357AC4214BFAF4241E050EA410E1CBF52EA430E02E0614650
:2067C0000020B0BD24423C441BD15FEA070EF6D0090302BF01460020AEF1140EB1FA81F71E
:2067E000AEEB070401FA07FE0C37C7F1200100FA07F7C8404EEA000E23EA455343F4801324
:020000040800F2
:20680000A2E733F00043B3FA83F704BFB2FA82FE77440B3FE41BB7F1200E2FBF02FA0EF3AE
:20682000BB40C7F1200E22FA0EFE38BF43EA0E03BA40641C82E750EA410E14BF52EA430E4E
:206840006FF000014FF4001717EB430F8ABF194617EB410FB5E74CEA05510020B0BDD4F1B6
:206860000104B4F120070FDAC4F12007520828BF42F0010210FA07F501FA07F7E1BF2A4300
:20688000E0403843E1400FE0352C98DCC7F1200452EA400220FA07F218BF42F0010231FAD4
:2068A00007F0A1400A43002172F1004250F1000051EB0C01B0BD0000F446400D40EAC12064
:2068C000490006D200F013F8004248BF6FF00040604700F00CF84FF0004188428CBF084636
:2068E00040426047400D40EAC12049000CD240F00040490DA1F58061491C05D4D1F11F0193
:2069000054BFC840C01770474FF000007047000030B585B004460D46208A4CF6FF7108407D
:20692000E98808432082A0894EF6F3110840A98808432989084369890843A081A08A4FF6FA
:20694000FF410840A9890843A08200A8FCF786F8144884420CBF0398029829681922504376
:20696000A28912044CBF49008900B0FBF1F16422B1FBF2F00001030902FB1311A3891B04DF
:2069800006D5C9003231B1FBF2F101F0070105E009013231B1FBF2F101F00F01084320819A
:2069A00005B030BD003801400029818912BF41F400514DF6FF7211408181704710B40B069F
:2069C0005B0F012401F01F0104FA01F1012B08BF0C3003D0022B0CBF10301430002A026815
:2069E00014BF114322EA0101016010BC7047C905C90D818070478088C005C00D704710B40D
:206A00000A06520F012301F01F0403FA04F4012A08BF828903D0022A0CBF028A828A224017
:206A2000090A03FA01F10088084022B1401E8041C043C00F00E0002010BC70472DE9F041F6
:206A40004FF0FF34DFF8DC552888DFF8DC65318800285BD04EF6EE62801A1FD041F2111275
:206A6000801A40F0878031B9284600F060FC042800F0848083E04EF6EE6081420BD128467F
:206A800000F055FC04287AD10021304600F06EFC042874D172E000F0A1F8F9E739BB002706
:206AA000DFF88865DFF888853088E988814208BF3C4624B2A7420BD0414600F062F8012865
:206AC00006D0B8F80010308800F0BBF8042856D17F1CB61C202FE7DB0021284600F046FC33
:206AE00004284CD1DFF8400500F021FCD0E74FF6FF70814207D1304600F019FC04283ED168
:206B000000212846C2E700F069F8C1E70029C2D04FF6FF70814205D1304600F008FC0428A6
:206B20002DD12BE00027DFF80455DFF804852888F188814208BF3C4624B2A7420BD041463F
:206B400000F01FF8012806D0B8F80010288800F078F8042813D17F1CAD1C202FE7DB0021B9
:206B6000304600F003FC042809D1DFF8B80400F0DEFB8DE700F032F8042800D10420BDE8FA
:206B8000F08170B504460D460126002000F039F8AB2816D0DFF88C1401EB8021DFF894240E
:206BA00002EB8020891C81420AD20288A24202BF30F8020C2880002602D0001F8142F4D356
:206BC000304670BD38B504460D4600F03AF8802803D12946204600F05BF832BD10B5DFF847
:206BE0004444204600F0A3FB042809D10021204600F0BCFB042804BFDFF82C0400F097FB6D
:020000040800F2
:206C000010BDDFF820140988DFF81C24128888B1012814D12AB94EF6EE6081420FD00120DB
:206C20007047002904D14EF6EE60824207D1F6E7AB207047002903D0002AF9D1EFE700202C
:206C4000704770B504460D460120FFF7DAFFAB281DD0DFF8D01301EB8026DFF8D81301EB11
:206C60008020864212D2316811F1010F0BD12946304600F07BFB042809D12146B01CBDE818
:206C8000704000F073BB361D8642ECD3802070BD2DE9F84304460F460020FFF7B2FF01289F
:206CA0000BD1DFF88083DFF880934EF6EE61404600F05CFB042808D02CE020B9DFF8688329
:206CC000DFF86093F1E7AB2024E039462046FFF7B8FF04281ED1DFF854732025DFF8506329
:206CE0003888A0420AD03146FFF74BFF012805D031883888FFF7A5FF04280BD1BF1C6D1EE2
:206D0000EED1484600F013FB042803D10021404600F02CFBBDE8F28330B583B0C34C45F2F2
:206D20005550208046F26660608047F27770A08048F68800E08049F6991020814AF6AA2037
:206D400060814BF6BB30A0814CF60740E0814CF6084020824CF6094060824CF60A40A082D4
:206D60004CF60B40E0824CF60C4020834CF60D40608300F0D1FAFFF761FEAF4D294620885E
:206D8000FFF7FFFEAB2804BF4FF425502880288841F28831401A43F6992180B2884224BF42
:206DA0004FF4255028802888A4490880A4490880A44D29466088FFF7E4FE10B14FF4AD7098
:206DC0002880288864384FF4D27180B2884224BF4FF4AD70288028889B4908809B490880CA
:206DE0009B4908809B4843F6982101809A4D2946E088FFF7C6FE08B1002028809748298848
:206E0000017000789649087001280CD1954801210170954801884FF6FD72114001809348F5
:206E20000188114001809248012101700DF106012089FFF7A6FE10B10020ADF8060001A90C
:206E40006089FFF79EFE10B10020ADF804008948BDF80610BDF8042002EB01410160864959
:206E6000006808600DF10201A089FFF78AFE10B10020ADF80200BDF80200000602D57F48B7
:206E80008021018000A9E089FFF77BFE10B10120ADF800007A48BDF8001001707949007896
:206EA000087000A9208AFFF76CFE10B11120ADF800007548BDF80010017074490078087070
:206EC00000A9608AFFF75DFE18B142F64420ADF800006F48BDF8001001806E490088088000
:206EE00000A9A08AFFF74DFE10B1B220ADF800006948BDF80010018068490088088000A9E5
:206F0000E08AFFF73EFE10B10120ADF800006448BDF80010017063490078087000A9208B7C
:206F2000FFF72FFE10B10320ADF800005E48BDF8001001705D490078087000A9608BFFF7A9
:206F400020FE18B14FF4AA70ADF800005848BDF80010018057490088088003B030BD10B54D
:206F6000044600F0D9F9FFF769FD21462F48C08818E038B5044600F0CFF9FFF75FFD2B4DD2
:206F8000210C2889FFF71EFEA1B26889BDE8344018E610B5044600F0BFF9FFF74FFD214646
:206FA00022488089BDE810400CE638B500F0B4F9FFF744FD1D4C324D2978E089FFF702FECE
:206FC000304829780170304D2978208AFFF7FAFD2E482978017031BD38B500F09DF9FFF793
:206FE0002DFD124C154D29882088FFF7EBFD144829880180154D29886088FFF7E3FD1448B5
:020000040800F2
:2070000029880180224D2988608AFFF7DBFD214829880180204D2988A08AFFF7D3FD1F4856
:2070200076E0000000F8000800FC00082402002062040020FEFB0008B80000204A040020E3
:2070400052040020BA000020C0000020C2000020560400202C04002028040020770400206D
:207060007A040020760400204E0100205001002059010020E8030020EC0300202A04002016
:207080005F0100208304002060010020840400204C01002054040020C4000020580400205B
:2070A00061010020850400206201002086040020520100205A04002038B500F02DF9FFF78E
:2070C000BDFC0C4C0C4D2978E08AFFF77BFD0B48297801700A4D2978208BFFF773FD09480E
:2070E00029780170084D2988608BFFF76BFD07480EE000BF240200206101002085040020C2
:207100006201002086040020520100205A0400202988018031BD000009490860704709496E
:207120000860704708490860704705484AF6AA210160704702484CF6CC410160704700009F
:207140000030004004300040083000404AB38B0707D0521E11F8013B00F8013B21D08B0701
:20716000F7D183071ED1103A07D330B4B1E83810103AA0E83810F9D230BC530724BFB1E83E
:207180000810A0E8081044BF51F8043B40F8043BD20724BF31F8022B20F8022B44BF0B7858
:2071A00003707047083A07D3B1E80810083A40F8043B40F804CBF7D25307E4E7F0B4254B16
:2071C00000241C804FF4807303804FF480644480202585804FF48045C580002686834FF442
:2071E0000056C683002707621B4F876047F6B767C7601A4F07611A4F4761002787618F61AC
:20720000184807800B804C8080208880CD808F83CE830F621448886047F6FF70C8604FF010
:2072200060400861114848618F611148078020201080012050809780D0809783D083176265
:207240000C48906044F62761D160106151619761F0BC70471C0400204981FFFF004052E0FF
:2072600000C0AD1F1A0400200080FFFF00C0FF1F1E040020D9B1FFFF30B4401AB2F9001025
:2072800000FB01F3B2F9041009B9002014E09469E5174843241855EBE0755069C117A94299
:2072A00002DC09DBA04207D31069B5EBE07F02DC02DB844200D320469061508893FBF0F0E7
:2072C0009169D38891FBF3F10918D068814204DA90688142B8BF0146084630BC7047000085
:2072E00062F30F2262F31F4200B5130096469446103928BFA0E80C50FAD85FEA417C28BF01
:207300000CC048BF40F8042BC90728BF20F8022B48BF00F8012B00BD00E00000DFF8A800F0
:20732000DFF8A8100160DFF8A8100160704738B505464FF4302000F051F8042815D1DFF8C9
:207340009440206840F0020020606560206840F0400020604FF4302000F040F8052804D026
:20736000216841F6FD721140216032BD70B504460D464FF4005000F031F8042810D1154E3F
:20738000306840F00100306025804FF4005000F025F8052804D0316841F6FE72114031602C
:2073A00070BD0D480168C90701D5012070470168490701D5022070470068C00601D50320D5
:2073C00070470420704700000420024023016745AB89EFCD102002400C20024010B5FFE76A
:2073E0000446FFF7DEFF03E02CB1FFF7DAFF641E0128F9D004B9052010BD00002DE9F04F69
:020000040800F2
:2074000085B0DFF8740A80680021DFF8700AFCF72DF900F097FC00F0FBFCFEF797FE4FF438
:207420009660FEF79FFEFEF7A0FE0028FBD0F9F75DFEFCF765FEFCF7A7FDFCF7FFFBFCF726
:207440000DFCDFF83C2ADFF83C1ADFF83C0AFFF7B5FEFEF7B9FCFEF721FDFCF737F9FCF720
:20746000F7FE4FF42550DFF8241A0880DFF8201A08804FF4AD70DFF81C1A0880DFF8181A2B
:2074800043F698220A80DFF8141A0880DFF8101A0880FFF74FFE4FF0C80BDFF808AADFF8A4
:2074A000088ADFF8085ADFF8086ADFF8087ADFF8084ADFF8089A1AE00021DFF8040AFBF7CB
:2074C00022FF072028700020FAF7DEFCDFF8F4090021416001600246D2E90001FAF754FAA7
:2074E000C820FEF73FFEDFF8E00900210170FEF74AFE012840F0E683FFF717FE0A20FEF7F7
:207500003FFED9F80000411CC9F80010DFF8BC090288DFF8BC090078012809D1A3783BB9E3
:207520000022DFF8B0391A8001236370626107E0B1FBFBF30BFB131313B9012808BF521C3E
:20754000DFF888391A806269521C6261A070E27890420BD0DFF8802912683AB9652905D393
:20756000FFF7FDFCDFF868090078E070D9F80000DFF868190968401A0B2813D3DFF86009BF
:20758000007878B9DFF85C09DFF85C1909780170DFF8540900210170FCF7B5FEDFF840093C
:2075A00001210170DFF844090068DFF84419097839B13968490404D4DFF81C190968782929
:2075C00001D2002000E0401CDFF820190860DFF82409006843F63521884203D26069C928B0
:2075E0000CD309E06078012808D16069C92805D3DFF804090121017000206070D9F800001F
:20760000032840F0A380FFF787FBDFF8F008DFF8F01809780170DFF8EC080068DFF8E418CE
:20762000496800EB0120DFF8DC18896800EB0140DFF8D018C96800EB0160DFF8CC1809683D
:207640000818DFF8C8180860DFF82C0800680190DFF8240840680290DFF81C18896803911A
:20766000019A120F41323270019A120E02F00F0241327270019A120D02F00F024132B270D4
:20768000019A120C02F00F024132F270019A120B02F00F0241323271019A120A02F00F02CE
:2076A00041327271019AC2F303124132B271019A02F00F024132F271020F41323272020ECD
:2076C00002F00F0241327272020D02F00F024132B272020C02F00F024132F272020B02F0C0
:2076E0000F0241323273020A02F00F0241327273C0F303124132B27300F00F004130F073C7
:20770000080F41303074080E00F00F0041307074080D00F00F004130B074080C00F00F0017
:207720004130F074080B00F00F0041303075080A00F00F0041307075C1F303104130B07588
:2077400001F00F004130F07500203076D9F80000642803D2DFF8B80700682061FAF71CFFD0
:20776000FBF7C2FFFAF702FCFCF7E3F9FCF791FA00F05BFBFCF799F82878032809D028780C
:20778000042806D0DFF88C0790F90000012840F0BD803868DFF88007DFF8F816B1F90010C1
:2077A0000180DFF87807B0F900000146DFF86827B2F900209042B8BF491C09B28A42B8BF25
:2077C0001146DFF858070180DFF85407B0F90000DFF85017B1F90010C1EB411141180A1156
:2077E00001EBD2614911DFF83C271180A16962890128A8BF4118501C4FF4007280B2904242
:020000040800F2
:2078000007D101F20010400ADFF81C170880002000216081A161DFF8FC0690F90000012802
:207820000CBF012100213B68DFF8002712885B0448BF002204D44FF416739A4238BF521C92
:20784000DFF8E8361A801A88642A01D200B90021DFF8DC261170117801292BD129780329E6
:2078600004D02978042901D0012831D14FF46040ADF8000010208DF8030003208DF8020080
:2078800000A94046FBF7B3F9DFF8880690F9000001281DD14FF400514046FBF71EFA4FF4AF
:2078A00080414046FBF719FA4FF400414046FBF714FA0DE04FF46040ADF8000018208DF840
:2078C000030003208DF8020000A94046FBF78FF9DFF8600600680A21B0FBF1F2DFF858368F
:2078E0001B68B3FBF1F18A4214D0DFF8EC15096881B9DFF8FC15097889B9FFF73AFBDFF895
:207900003806DFF830160968016003E0DFF8140600210180DFF8C0050068002852D1D9F8A4
:207920000000B0F5167F4DD9DFF810060078DFF810160978884207D1DFF808060078DFF82E
:2079400008160978884201D0FFF72FFBDFF8FC050088DFF83C150988884217D1DFF8F00536
:207960000088DFF83C15098888420FD1DFF8E4050088DFF8E4150988884207D1DFF8DC0519
:207980000088DFF8DC150988884201D0FFF724FBDFF8D0050078DFF8D015097888420FD14B
:2079A000DFF8C8050078DFF8C8150978884207D1DFF8C0050088DFF8C0150988884201D0D8
:2079C000FFF77AFBDFF84C0590F9000070B94FF400514046FBF77FF94FF480414046FBF762
:2079E0007AF94FF400414046FBF775F9DFF88C0500884FF42F71884203D2401CDFF87C1574
:207A00000880DFF878050088DFF87415098800EB800291420ADA652808D3DFF868150978B0
:207A2000484300EB8000DFF860150880DFF85805008840F6AD51884204D3DFF84C0540F68D
:207A4000AC510180FEF744FADFF840050088DFF848140988DFF838251268914205D347F27B
:207A60003051884202D2401C00E00020DFF81C1508804FF40041DFF81C05FBF721F901284A
:207A800004D1617901291CBF0021A1816071BAF8001001280EBF41F008004FF6F770084039
:207AA000AAF80000A089401CA08180B2B0F5966F04D210214046FBF710F903E01021404680
:207AC000FBF709F94FF40041DFF8C804FBF7F8F8012803D1386820F400603860D9F800002F
:207AE0004FF49671884204D2DFF8AC04BAF800100180DFF8A80400780146C92838BF491C43
:207B0000DFF894040288BAF800000AB900B10021DFF88834197082421CBFDFF87C1408807B
:207B2000197819B1642901D0C82904D118B10C21E020FCF755FFDFF86804008842F2107109
:207B4000884203D2401CDFF858140880DFF8500400884FF41671884234BF4FF49670642058
:207B6000DFF840140988042923BFDFF83C140988491C0021DFF830241180E188491CE18011
:207B800089B281420DD3DFF824040078DFF820140978884205D10C21FF20FCF721FF0020E5
:207BA000E080DFF810040078012806D120214046FBF791F80020207109E02079401C2071A0
:207BC000C0B2C92803D320214046FBF786F84FF480714046FBF774F8012807D04FF4004199
:207BE000DFF8B003FBF76CF8012808D1DFF8C40301210170DFF8C003002101602EE0DFF871
:020000040800F2
:207C0000B8030068401CDFF8B0130860012804BF00212170AE490978C1B9C9281ED3DFF89A
:207C2000940300210170B2480078B8B9C1480068C1490968884211D0217879B9FFF799F94E
:207C400001202070BC48BB490968D6E7012905D1DA4909880BFB01F18142E0D3D848007883
:207C600070B9D848008858B1D74800210180D7480180FCF704FAD64800210180D54801807A
:207C80009548006800280CBFD348D4480088CD490988090503D52189814238BF0846C7499E
:207CA0000880088820810BFB00F0D9F80010CC4A1268891A884205D2BAF8000040F010006E
:207CC000AAF800002878022807D005283FF4F4AB072814D008281BD009E4F9F788FC386833
:207CE0004FF40C7108427FF402ACFBF7D3FC4FF4FA60FEF741FA03202870FFF7F8BBFEF772
:207D000034FA01287FF4F3ABFCF7B9F90120F3E7386840F67E71084004286B480CD100781A
:207D200006280BD2401C6849087001202870386820F00400386001E000210170FCF79FF9B0
:207D4000FFF7D5BB10B582B001210C20FAF7CCFE01210120FAF7C8FE0121A248FAF7C7FFE0
:207D60000121A148FAF7C3FF8A4C2046FAF7F4FE4FF480712046FAF7B0FF4FF400712046D2
:207D8000FAF7ABFF4FF480612046FAF7A6FF00A8FAF78EFF4FF4F850ADF8000010208DF81D
:207DA000030003208DF8020000A92046FAF71FFF3D4C2046FAF7D0FE4FF400512046FAF75F
:207DC0008AFF4FF480412046FAF785FF4FF400412046FAF780FF4FF46040ADF80000102029
:207DE0008DF8030003208DF8020000A92046FAF7FEFE40F63C60ADF8000001208DF8020036
:207E000010208DF8030000A92046FAF7F0FE13BD80B545F25550FFF77FF90220FFF77FF9DD
:207E20007F20BDE80240FFF77DB910B46F48B0F90000411E40F6A92289B2914238BF40F6D1
:207E4000AA206B49B1F9002002F1C8048442B8BF02F1C80000B200F1C8049442B8BFA2F1D4
:207E6000C80000B20128A8BF4FF48040614A10801088088010BC7047E8F7FF1F0010000802
:207E80001C030020D4020020F8020020B80000204A040020BA0000202C040020C000002043
:207EA000C20000204E010020000C01406804002064030020BC030020E0000020C00300204F
:207EC000002C01409803002002000020220400207704002024040020E0030020D803002031
:207EE0005D0100206A04002071040020F40300207F040020CC0300206F0400205A0100202A
:207F0000590100203800002018E000E0FC030020C40300206E0400209400002096000020B5
:207F20009A00002038040020480400202604002072040020E8030020EC030020830400201E
:207F40005F01002084040020600100205204002056040020540400204C0100205804002027
:207F6000C4000020850400206101002086040020620100205A040020520100202E04002082
:207F8000480100205C0100203601002050040020DC030020000801405001002063010020F3
:207FA000560100205C0400205E0400206B0400207504002058010020C80300204404002054
:207FC0007B0400202A0400203C0400203A0400201C0400201A040020540100204A01002098
:207FE000E403002000043000000230004004002018040020A60300207047FEE7FEE7FEE745
:020000040800F2
:20800000FEE770477047704741480168490700D4704700B581B06FF004010160F9F796FF59
:2080200060B13C480078032806D0042801D0062804D1FDF7DAFD01E0FCF7D6F801B000BD57
:2080400000B581B080213448FBF7A1F94FF40070FBF759FB3148006865280CD3012080F3B7
:2080600013882F48016801F4E0612E4A11430160BFF34F8FFEE701B05DF804EBFFF755B8B5
:2080800000B581B001212448FBF780F901B05DF804EBF9F717BF70B5234801210170234CB4
:2080A00040F225512046FEF7AAFCA0B120481B49096801601F48002101702046FEF79BFC3D
:2080C0001D490A781D4BD054501C0870C0B2402824BF0020087040F2277529462046FEF75B
:2080E0008EFC98B1164E30781649415C2046FEF77EFC3078401C307013490978C0B2884213
:2081000004D1002229462046FEF758FC70BD00000024014068040020002C0140C0030020DC
:208120000CED00E00400FA055E01002000380140D80300205D01002071040020E401002058
:208140006B040020A0020020750400202648016841F0010101604168244A11404160016858
:20816000234A11400160016821F480210160416821F4FE0141604FF41F018160016821F440
:20818000803101601B490A6842F010020A600A68920892000A600A6842F002020A60416886
:2081A000416041684160416841F480614160416821F47C114160416841F46011416001682F
:2081C00041F08071016001688901FCD54168890889004160416841F002014160416801F0DC
:2081E0000C010829FAD17047001002400000FFF8FFFFF6FE002002402DE9F04100F10801E1
:20820000026801EB8202406800F001034008400002EB80004FF0000CE646002401250CE046
:208220001CF8018BBE4206D006F8018B641C24B2002CF7D40125BE4212D1824201D1BDE8AD
:20824000F08152F8046B03B14E4452F8047BBF19F1E7D1F800C08C44091D51F804EBE64454
:20826000F445F6D065B11CF9014B002506E0D1F800C08C44091D51F804EBE644F445F6D09D
:20828000002CCDD424B2002CD4D4BE4218BFF4451EBF1CF8018B06F8018B641EF2D1CAE75A
:2082A00010B5084979441C31074C7C441A34A14206D0081D0A68511888470146A142F8D1C2
:2082C00010BD00BF080000003000000013BEFFFF2803000064010020000000001DFFFFFF41
:2082E00002000000020000004001000084000000000000206401000000F009F8002801D046
:20830000FFF7CEFF0020FFF779F800F002F80120704780B500F002B800BF000007463846E8
:2083200000F002F8FBE7000080B5C046C046024A11001820ABBEFBE7260002000148804718
:20834000014800474D8100084D830008C046C046C046C046FFF7D0FFFFF74EBEFFF74DBEFF
:20836000FFF74CBEFFF74BBEFFF74ABEFFF749BEFFF748BEFFF747BEFDF708BFFFF7FEBF9E
:20838000FFF7FEBFFFF7FEBFFFF7FEBFFFF7FEBFFFF7FEBFFFF7FEBFFFF7FEBFFFF7FEBF45
:2083A000FFF7FEBFFFF7FEBFFFF7FEBFFFF7FEBFFFF7FEBFFFF7FEBFFFF7FEBFFFF7FEBF25
:2083C000FFF7FEBFFFF720BEFFF7FEBFFFF7FEBFFFF7FEBFFFF7FEBFFFF7FEBFFFF730BEB3
:2083E000FFF74EBEFFF7FEBFFFF7FEBFFFF7FEBFFBF725BCFFF7FEBFFFF7FEBFFFF7FEBF76
:020000040800F2
:20840000FFF7FEBFFFF7FEBFFFF7FEBFFFF7FEBFFFF741BEFFF7FEBFFFF7FEBFFFF7FEBF82
:20842000FFF7FEBFFFF7FEBFFC0002040506FB000001DF0003BC02BC02E400040200008005
:2084400002FD000003AF0000FAE90007FD00FD00B2005E01E7000001FA00003CFD0001B0AA
:2084600004EE0002E70301FA00002DF200100102030401020304060708090204060801F7B6
:20848000000001FD0003AC0D0001F600131A085E01AC0D3C00442A0200020054016009DC96
:2084A00005FD010005FC0103110103FAFFFFFFFFFFFFFFFFFFFFFFFFFFFFFFFFFFFFFFFFB9
:2084C000FFFFFFFFFFFFFFFFFFFFFFFFFFFFFFFFFFFFFFFFFFFFFFFFFFFFFFFFFFFFFFFFBC
:2084E000FFFFFFFFFFFFFFFFFFFFFFFFFFFFFFFFFFFFFFFFFFFFFFFFFFFFFFFFFFFFFFFF9C
:20850000FFFFFFFFFFFFFFFFFFFFFFFFFFFFFFFFFFFFFFFFFFFFFFFFFFFFFFFFFFFFFFFF7B
:20852000FFFFFFFFFFFFFFFFFFFFFFFFFFFFFFFFFFFFFFFFFFFFFFFFFFFFFFFFFFFFFFFF5B
:020000040800F2
:020000040800F2
:20F800000000FFFF00008888402955553B016666000099999805AAAA0000BBBB010007CC52
:20F82000110008CC442A09CCB2000ACC000099999905AAAA010088880000888800009999A1
:20F840009F05AAAA0100888800009999A205AAAA0000888801008888010007CC080008CCA1
:20F86000010007CC110008CC00009999B105AAAA00009999B505AAAA000088880000999911
:20F88000BB05AAAA01008888000088880100888800009999C005AAAA0000888801008888B6
:20F8A00000009999CD05AAAA00009999D205AAAA0000888801008888000088880000999930
:20F8C000D605AAAAFFFFFFFFFFFFFFFFFFFFFFFFFFFFFFFFFFFFFFFFFFFFFFFFFFFFFFFF15
:20F8E000FFFFFFFFFFFFFFFFFFFFFFFFFFFFFFFFFFFFFFFFFFFFFFFFFFFFFFFFFFFFFFFF28
:20F90000FFFFFFFFFFFFFFFFFFFFFFFFFFFFFFFFFFFFFFFFFFFFFFFFFFFFFFFFFFFFFFFF07
:20F92000FFFFFFFFFFFFFFFFFFFFFFFFFFFFFFFFFFFFFFFFFFFFFFFFFFFFFFFFFFFFFFFFE7
:20F94000FFFFFFFFFFFFFFFFFFFFFFFFFFFFFFFFFFFFFFFFFFFFFFFFFFFFFFFFFFFFFFFFC7
:020000040800F2
:00000001FF
